:100000000264F702683B0000000000026155000036
:1000100000000002689900000000003200000000AB
:10002000000000022C6A000000000002628B000049
:1000300000000000000000000000000000000000C0
:100040005052343032207665722E3133312E312EBB
:1000500031204864773A482032342D31302D303504
:100060002032333A3134202075F00612011E22125C
:100070005ECC75F00612011E125ED12212006F12C4
:10008000006812006F12006812006F120068120000
:100090006F12006812006F75F01812011E22125EB6
:1000A000CC75F04B12011E125ED122755004122540
:1000B000CF1225E5125ECC75F0C812011E125ED17A
:1000C000227550051225CF1225E512009E75F01EEF
:1000D00012011E12009E227550071225CF1225E52F
:1000E000120088227550061225CF1225E512008EC7
:1000F0002212007C12007C221200E41200E41200A2
:10010000E422C2A1C25312006F75F01212011ED276
:10011000A1C2532212006F75F01212011E22128624
:1001200096201807C0F01284F7D0F0D5F0F02270B6
:1001300004A23EB322C0E01412013ED0E022C0E08F
:10014000030303540F28F8D0E0C0E0540704F5F08F
:10015000E213D5F0FCD0E0227003D3802830E7030F
:10016000C3802223F9C3137004A23E801814C0E098
:10017000030303540F247AF8D0E0540704F5F0E2A7
:1001800013D5F0FCE992E022C0E024B8F8E21201B5
:10019000584004D0E0C322D0E024CEF5827400346D
:1001A00000F583E01201A82220E702C322C2E7C0C3
:1001B000E0C2E0700AA23EB3D0E030E001B322B466
:1001C0007E03C380F3B40204A22580ECB40404A22D
:1001D0002680E5B40604A22780DEB40804A20380CA
:1001E000D7B40A04A20E80D0B40C0AE5714572C3DC
:1001F0006001D380C3B40E0512613780BBB4100711
:10020000A2597258B380B1B41206A258822880A8AD
:10021000B41406A258B028809FB41604A25980983E
:10022000B418077400126E74808EB41A0774011229
:100230006E748084B41C087402126E740201B8B427
:100240001E087403126E740201B8B42008740412FC
:100250006E740201B8B422087405126E740201B8FB
:10026000B424087406126E740201B8B42608740728
:10027000126E740201B8D0E0C322123227E5686022
:1002800013B401051202AC8008B402051202C68044
:10029000007568001284F7E5735440600B20A808CD
:1002A000305005C25012856D126CC322C23ED2700E
:1002B000C2AF75186075190F751AFA120A3F757971
:1002C00003C240C24322D23EC270C2AF75187075DD
:1002D000190F751AFA120A3F75790322C2B612670E
:1002E000E475370074031249E9E51E1249E9E51F78
:1002F0001249E974571249E9120305E5371249E931
:100300003099FDD3227881E6232354031249E978FA
:1003100082E630E402240A540F1249E97881E6C4E7
:10032000540375F00AA4F5F0E6540F25F01249E9DC
:100330007880E6C4540375F00AA4F5F0E6540F255E
:10034000F01249E9787FE6C4540775F00AA4F5F085
:10035000E6540F25F01249E9787EE6C4540775F09B
:100360000AA4F5F0E6540F25F01249E97882E60375
:10037000C454071249E92275F0321286AEB2B512A2
:1003800086AEB2B5D5F0F322D2A3C251D2A2C254E6
:10039000C2A1C253D2A4C252C2A0125ECC12037731
:1003A000D2A0125ED1120377C2A0125ECC120377E4
:1003B000D2A0125ED1120377C2A0125ECC120377D4
:1003C000D2A0125ED11203771203771203771203C1
:1003D0007712037722C0F075F0DCD5F005B2B512C4
:1003E00005A3C0F0120596D0F030E7EED0F022AAB7
:1003F000F01203D5E532652FF5F0E533653045F0B1
:10040000600C1204E5852F328530331203D51205B6
:100410005B1203D51205831203D51204F28AF0226F
:10042000AAF01203D5E532652FF5F0E533653045C6
:10043000F0600C1204E5852F328530331203D5129B
:1004400005471203D51205831203D51204F28AF070
:1004500022AAF01203D5E532652FF5F0E5336530B9
:1004600045F0600C1204E5852F328530331203D538
:100470001205178AF022AAF01203D5E532652FF58E
:10048000F0E533653045F0600C1204E5852F3285C8
:1004900030331203D51204FF8AF022C0F075F00841
:1004A00033C297928300D297D5F0F5D0F022C0F0F6
:1004B00075F008C297D29700A28233D5F0F5D0F03C
:1004C00022D2B7D297D283D282D2842212049BE561
:1004D0003033E52F3312049BC3E5303312049BE520
:1004E0003112049B221204C1C28474531204CCD270
:1004F00084221204C1C28474581204CCD284221201
:1005000004C1C28474541204CCE412049B1204AEDD
:10051000F608D9F9D284221204C1C2847454120498
:10052000CCE412049B1204AEF208D9F9D284221250
:1005300004C1C28474541204CCE412049B1204AEAD
:10054000F0A3D9F9D284221204C1C28474841204A3
:10055000CCE612049B08D9F9D284221204C1C284C9
:1005600074841204CCE212049B08D9F9D2842212BA
:1005700004C1C28474841204CCE012049BA3D9F990
:10058000D284221204C1C28474831204CCD2841295
:10059000869612869622C284745712049B1204AE69
:1005A000D2842275F06412059620E50430E301221E
:1005B000C2AFB2B51286AEB2B51286AED5F0E712B2
:1005C000038880FBD283D282D297D2B7D284B2B5CD
:1005D00075F002128696D5F0FAC2B7B2B575F00280
:1005E000128696D5F0FAD2B7B2B5227920752F01CE
:1005F0007530037531E09000E41203D51204E51262
:1006000003D512052F7900752F017530047531005F
:100610009001041203D51204E51203D512052F79B7
:10062000E0752F017530057531009002041203D575
:100630001204E51203D512052F852F32853033229F
:10064000752F017530DB7531001203D51208DB758B
:1006500032FF7533FF22AE83AD8290DB007F2074C2
:1006600004F9747CF8752F0185833085823112047A
:1006700076787CE66E702508E66D702008E6601AD4
:10068000B4FF028013167404F9747CF8752F018589
:100690008330858231120420C322D322A3A3A3A3D3
:1006A000DFBD80F490DB007F207404F9747CF87562
:1006B0002F01858330858231120476787CE66E7056
:1006C0000908E66D700408E6FC22A3A3A3A3DF0AD1
:1006D0007CFF2290DB007F207BFF7404F9747CF8A0
:1006E000752F01858330858231120476787CE66E21
:1006F000702C08E66D702708ECB4FF0D787C76FF4F
:100700000876FF0876FF0874FFF67404F9747CF825
:10071000752F01858330858231120420C322BBFFEF
:1007200010787CE6B4FF0A08E6B4FF05C374209F86
:10073000FBA3A3A3A3DFA3BBFF02D322EB2323547A
:10074000FC2400F5827583DB50020583787CEEF68D
:1007500008EDF608ECF608E4F67404F9747CF87514
:100760002F01858330858231120420C322758300D6
:1007700075F08E752F02858330753100C0F0C0830F
:100780001203D51208DBD0830583D0F0D5F0E475D1
:10079000830075F0DA752F03858330753100C0F062
:1007A000C0831203D51208DBD0830583D0F0D5F0C7
:1007B000E47532FF7533FF2275830075820075F092
:1007C0008EC0F0C082C083752F02858330753100E2
:1007D0001203D51204E5D083D082C082C083752F66
:1007E000008582307531001203D5120583D083D085
:1007F0008205830582D0F0D5F0C77583007582002D
:1008000075F0DAC0F0C082C083752F038583307520
:1008100031001203D51204E5D083D082C082C08398
:10082000752F018582307531001203D5120583D0F2
:1008300083D08205830582D0F0D5F0C77532FF756D
:1008400033FF2275830075820075F08EC0F0C08280
:10085000C083752F008583307531001203D51204D3
:10086000E5D083D082C082C083752F028582307527
:1008700031001203D5120583D083D082058305820F
:10088000D0F0D5F0C775830075820075F0DAC0F03E
:10089000C082C083752F018583307531001203D566
:1008A0001204E5D083D082C082C083752F03858275
:1008B000307531001203D5120583D083D0820583B1
:1008C0000582D0F0D5F0C77532FF7533FF221204D0
:1008D000C1C28474501204CCD284221204C1C284D6
:1008E00074811204CCD284221204C1C28474841292
:1008F00004CCE812049BD9FAD28422F879001203BE
:10090000D51208E8EAC0E085822F85833075310072
:100910001203D5120583D0E0FA0583DAE77532FFBA
:100920007533FF221204C1C28474541204CCE41241
:10093000049BE4C0E01204AED0F025F0D9F5D284D7
:10094000227583007582028006758300758200E43B
:1009500075F08D85822F858330753100C082C0830C
:10096000C0F0C0E01203D51204E51203D5790012DD
:100970000924D0F025F0D0F0D083D0820583D5F0C3
:10098000D285822F858330753100C0E01203D512E5
:1009900004E51203D57920120924D0F025F0753230
:1009A000FF7533FF2275830075820380067583000F
:1009B000758201E475F0DA85822F85833075310008
:1009C000C082C083C0F0C0E01203D51204E5120358
:1009D000D57900120924D0F025F0D0F0D083D08250
:1009E0000583D5F0D27532FF7533FF05E02275839C
:1009F0000075F000752F00858330753100C0F0C0A0
:100A0000831203D51208DBD0830583D0F0D5F0E440
:100A10007532FF7533FF75830075F0DA752F018528
:100A20008330753100C0F0C0831203D51208DBD0CB
:100A3000830583D0F0D5F0E47532FF7533FF225380
:100A4000560F53550F5318F053190FC2AFE55523E6
:100A500024ADF8E5184519F608A61A055553550FA3
:100A6000E555B55605055653560FD2AFC3E5559516
:100A7000565002241024F4500375600022E556B548
:100A800055057400780022C33324ADF8E6C0E008B1
:100A9000E6F8D0E02253550F53560FC2AFE556B5D6
:100AA0005504D2AFD322055653560FD2AFC32230CE
:100AB0000C597881E6540FC0E0E6C4540375F00A7F
:100AC000A4D0F025F0FD7882E630E402240A540F29
:100AD000FE901A007F3C7404F97400F8752F0185AC
:100AE00083308582311204517800E26D701708E27C
:100AF0006E701208E2C42354E0F5F07882E6541FC9
:100B000045F0F68006A3A3A3A3DFCB221267E4126D
:100B10000AAF1267F3FEAFF07DFF0DED30E7012263
:100B2000D25C75F004A424E4F582E5F03400F5838A
:100B3000C082C083787CE0F6A308E0F6A308E0F664
:100B4000A308E0F6D083D082787C868308868278FA
:100B50007CB6FF0708B6FF03020BD2C3E58233F56C
:100B600082E58333F583E58224E0F582E58334056D
:100B7000F583787EE6705B08E66057FB7402F974D3
:100B80007CF8752F01858330858231120476A3A30A
:100B9000787CE60856B4FF03020BD2787C86F053CB
:100BA000F07F08E6C39EC5F09F401E7025E5F0600B
:100BB00018BD001E203E1B787CE6A2E720E713E567
:100BC000F024FA400DD26B8009787CE6A2E7925CB3
:100BD000DBAABD00028028ED14C0E0030303540F1C
:100BE000247AF8D0E0540704FB7400D333DBFD30E3
:100BF0005C05FBE24B8004F4FBE25BF2020B1AB2F1
:100C00005C128546406F202F6C206F6920190B20E5
:100C10003D05305C608003205C5B305C3D203D3AEC
:100C200078B7E2702F206A2178B5E2602D1264B1A6
:100C30006028F5F0E5F0543F4400C2AF7518C07568
:100C40001909F51A120A3F80051264B1600C78B5D3
:100C5000E278B7F2D26BD26A801BC26BC26AA25C26
:100C6000923D400B303E0E120C7812424A80062014
:100C70003E03120C92020B1AC23ED270C2AF75181C
:100C80006075190F751AE0120A3F757903C240C2E8
:100C90004322D23EC270C2AF75187075190F751A13
:100CA000E0120A3F7579032212049BE53033E52FE9
:100CB0003312049BC3E53033D2E012049BE53112BA
:100CC000049B221204C1C2847454120CA8E41204BE
:100CD0009B1204AEF608D9F9D284221204C1C28450
:100CE0007484120CA8E612049B08D9F9D2842290CD
:100CF000FC00752F04753000753100C082C083750B
:100D00004AFA1203D51204E5852F67853066790803
:100D1000787C1203D5120CC3120F43D083D082709B
:100D200044C082C08378808683088682120D9C40EE
:100D300024787E8683088682120D9C4018120DBB93
:100D4000E582600AE564B5660CE565B56707D083A2
:100D5000D082020D77787EE6249AF6120F8612036F
:100D600088D083D0820530E5307002052FA3E5825C
:100D700045837087120D7E7532FF7533FF22787EB2
:100D800076000876007880760008760008760008FD
:100D90007600756704756600120F6222C082C083F8
:100DA000E5822400F582E5833480F5834005D08315
:100DB000D08222D083D08290000022E58275F00894
:100DC000A4F582E5F0C58375F008A42583F583E5D5
:100DD000F03404F565E5822400F582E5833400F5FE
:100DE000835002056585836422120388D083D082F4
:100DF00022C082C083120F1C70EF787E8683088623
:100E000082120D9C40E3120DBB1211FD787C76001E
:100E10007880E518F608E519F6087600087600747B
:100E200008F9747CF885652F85833085823112043A
:100E3000207404F97480F885652F858330858231AC
:100E400012047675F004787C7980E66760028099F8
:100E50000809D5F0F5120F23787E8683088682A3D1
:100E6000120D9C787EA68308A682788086830886E9
:100E700082120D9C787EE66583706208E66582705A
:100E80005CC065C064C082C083120DBB7408F97475
:100E900084F885652F8583308582311204767888C1
:100EA00076C0087657087600087600D083D082E5B1
:100EB00082241EF58250020583120D9CC082C083DD
:100EC000120DBB7408F97484F885652F858330850D
:100ED0008231120420D083D082D064D0657880A67D
:100EE0008308A682C067C066856567856466120F41
:100EF00062D0E0D0F0B56609C5F0B567028018C5CC
:100F0000F0C067C06685F067F566787EE62499F6DE
:100F1000120F86D066D067D083D08222120F2312A0
:100F20000F432285672F8566307531001203D51275
:100F300004E57908787C1203D5120CC3852F32851D
:100F40003033227881E6182618261826182455668C
:100F5000700F7881E6186618661866186618649926
:100F60006622120F69120F86227881E6182618264B
:100F70001826182455F67881E6186618661866183B
:100F800066186499F62285672F85663075310012E0
:100F900003D51204E51203D57908787C120CDB1214
:100FA00003D51205831203D51204F2852F32853042
:100FB0003322120F1C7030787EE6C0E008E6C0E0F5
:100FC000088683088682C3D0E09582F582D0E095BA
:100FD00083F58350104582600CE5822400F582E59C
:100FE000833480F583C322900000D322C2B6120F4F
:100FF000B2E433C0E075370074031249E9E51E120C
:1010000049E9E51F1249E974531249E9D0E0124950
:10101000E974001249E974001249E9E5831249E9CB
:10102000E5821249E9E5371249E93099FD22C2B655
:10103000E5356004F4FF8004FF120D7E75370074FF
:10104000031249E9E51E1249E9E51F1249E9745600
:101050001249E9EF1249E9E5371249E93099FD22D1
:101060007401C0E0787C75F008E4F608D5F0FBD098
:10107000E0D322120FB240E860E8788086830886C9
:1010800082121086C322C082C083E58275F008A454
:10109000F582E5F0C58375F008A42583F583E5F0B6
:1010A0003404F565E5822400F582E5833400F58398
:1010B000500205657408F9747CF885652F858330C6
:1010C000858231120476D083D08222120FB27F083B
:1010D0005005120D7E7F00787E8657088658088658
:1010E0005908865AC2B675370074031249E9E51EDD
:1010F0001249E9E51F1249E974541249E9E535122C
:1011000049E9EF1249E9E535603CE55A6558F5F0E3
:10111000E559655745F0600B855A82855983121051
:10112000868003121062855A82855983A3120D9C12
:1011300085825A858359787C75F008E61249E9085A
:10114000D5F0F8D535C4E5371249E93099FDC32209
:10115000E5357007C2AF120FB25005E535F4800CCB
:101160007880A65908A65A120F62E535D2AFC0E0C2
:10117000C2B675370074031249E9E51E1249E9E564
:101180001F1249E974551249E9D0E01249E9E537DF
:101190001249E93099FDD322C2B6753700740312A3
:1011A00049E9E51E1249E9E51F1249E97458124957
:1011B000E97420232354FC041249E974201249E9FC
:1011C00090DB007F207404F9747CF8752F0185830F
:1011D00030858231120476787CE61249E908E612FD
:1011E00049E908E61249E908E61249E908A3A3A378
:1011F000A3DFD2E5371249E93099FDD3221267E423
:101200007882E630E402240A540FC4F97881E6C4F7
:10121000540375F00AA4F5F0E6540F25F0C3134902
:10122000787DF67881E692E754C0F9787FE6C45479
:101230000775F00AA4F5F0E6540F25F049F9788017
:10124000E6C4540375F00AA4F5F0E6540F25F0F552
:10125000F0787EE654702345F0787FF6787EE9F6E4
:101260002222303FFD125ECC75F00612011E125E86
:10127000D175F01412011EE53FC23F22E422787CB2
:101280007910E6B5F0070805F0D9F7E422740122D9
:10129000C0E0787C7910F60805E0D9FA7410F9748A
:1012A0007CF8752F037530DB753100120420741043
:1012B000F9747CF8752F037530DC75310012042049
:1012C0007410F9747CF8752F037530DB75310012DA
:1012D0000476D0F0C0F012127E701E7410F9747C87
:1012E000F8752F037530DC753100120476D0F0C02C
:1012F000F012127E7003D0F022D0F022E51DC0E083
:10130000121290D0F07006E5F0F412129022785587
:1013100074FFF212142AC20C1209AD6001221205E8
:10132000EB7401F97455F8752F017530037531A010
:101330001204517410F9748AF8752F017530037511
:1013400031C01204517410F9749AF8752F01753078
:10135000037531D01204517402F97467F8752F01C6
:101360007530CE7531001204517416F974B8F875E1
:101370002F017530CE7531C012045178B89000CE6F
:1013800075F016E2F008A3D5F0F97416F974B8F800
:10139000752F017530037531A11204517408F97469
:1013A00000F8752F017530D27531001204517800A4
:1013B0009002F775F008E2F008A3D5F0F9D20CE43A
:1013C00022797C776509E4A23E92E0A23D92E7F79C
:1013D000097404F9747CF8752F0275308E7531002C
:1013E00012042022D23EC270D23D22C26F7404F990
:1013F000747CF8752F0275308E7531001204767882
:101400007CB665E008E6D26FA2E0923EB39270A28D
:10141000E7923D787C76FF7401F9747CF8752F02B1
:1014200075308E7531001204202278B875F016E4FC
:10143000F208D5F0FB74FF78C0F278C1F222E8C060
:10144000E07862E2F56CD0E0F822E8C0E07863E290
:10145000F56CD0E0F822E8C0E07864E2F56CD0E00A
:10146000F82275F00384B40104741A8017B40204DE
:1014700074228010B40304742A8009B404047442F2
:101480008002741A227403F9745FF8752F007530A6
:101490008C7531E5120451785FE21214627862F2C1
:1014A0007860E21214627863F27861E21214627872
:1014B00064F2785FE224FD9208E224E2920974016A
:1014C000F9745EF8752F0075308C7531E212045195
:1014D000785EE224FD9206E224E29207227403F988
:1014E000745FF8752F0075308C7531E51203EF7459
:1014F00001F9745EF8752F0075308C7531E21203B6
:10150000EF22797C774809774E0977830977A074B1
:1015100004F9747CF8752F0075308D753120120434
:10152000207404F9747CF8752F0275308D753120A4
:10153000120420227404F9747CF8752F0075308D24
:10154000753120120476797EE7648322E4A21E922C
:10155000E0A21F92E1A22092E2A20192E3797CF73D
:101560007401F9747CF8752F0075308C7531E812B0
:101570000420227401F9747CF8752F0075308C7585
:1015800031E8120476797CE7A2E0921EA2E1921F74
:10159000A2E29220A2E3920122797CE4A22B92E0C3
:1015A000A22C92E1A22D92E2A21692E392E492E59D
:1015B000A22F92E692E7F709E4A22E92E0A23092DF
:1015C000E1A23192E2A23292E3A23492E6A23592F3
:1015D000E7F709E4A23692E0A23892E2A23992E358
:1015E000A23A92E4A23B92E5A23C92E7F709E573A6
:1015F000F77404F9747CF8752F0075308C7531EC34
:10160000120420797CE574F4F709E575F4F709E52F
:1016100076F4F77403F9747CF8752F0075308C75C7
:1016200031E9120420227404F9747CF8752F0075D6
:10163000308C7531EC120476797CE7A2E0922BA213
:10164000E1922CA2E2922DA2E39216A2E6922FA2A0
:10165000E709E7A2E0922EA2E19230A2E29231A243
:10166000E39232A2E69234A2E7923509E7A2E09231
:1016700036A2E29238A2E39239A2E4923AA2E5922B
:101680003BA2E6A2E7923C09E7F5737403F9747C88
:10169000F8752F0075308C7531E9120476797CE786
:1016A000F4F57409E7F4F57509E7F4F57622797C29
:1016B000F77401F9747CF8752F0075308C7531E47E
:1016C000120420227401F9747CF8752F0075308C97
:1016D0007531E4120476797CE7227401F9744FF8CD
:1016E000752F0075308C7531FC1203EF227401F9EF
:1016F000744FF8752F0075308C7531FC120451222F
:10170000784FE270067850F208F22275F000303A15
:101710000475F03CA4AAF075F008A4FBACF0EA75DF
:10172000F008A42CFAC374FD9BFB74FF9A7850F266
:10173000EB08F2227401F97452F8752F0075308DA0
:101740007531001203EF227401F97452F8752F00FD
:1017500075308D753100120451227402F97470F8DD
:10176000752F0075308C7531FD1204517402F974B7
:1017700072F8752F0075308D753101120451227485
:1017800002F97470F8752F0075308C7531FD1203F5
:10179000EF7402F97472F8752F0075308D75310190
:1017A0001203EF227401F97456F8752F0075308C0E
:1017B0007531F01203EF7401F97457F8752F007545
:1017C000308C7531F41203EF7401F97458F8752FE9
:1017D0000075308C7531F61203EF7401F97459F805
:1017E000752F0075308C7531F21203EF227401F9F8
:1017F0007456F8752F0075308C7531F012045174E1
:1018000001F97457F8752F0075308C7531F4120496
:10181000517401F97458F8752F0075308C7531F6D4
:101820001204517401F97459F8752F0075308C75D4
:1018300031F2120451227401F97438F8752F0075D1
:10184000308C7531F81204207401F97439F8752F51
:101850000075308C7531FA1204207401F9743AF86D
:10186000752F0075308C7531FB120420227401F93C
:101870007438F8752F0075308C7531F81204767451
:1018800001F97439F8752F0075308C7531FA12042E
:10189000767401F9743AF8752F0075308C7531FB48
:1018A000120476227402F9741EF8752F0075308CBC
:1018B0007531E0120420227402F9741EF8752F00AD
:1018C00075308C7531E012047622E576540260039F
:1018D000756B03789D7980AA6B80021819E7F5F083
:1018E00066540F700E18E7C4F5F066540F7004DAF2
:1018F000EAE422E6540FC5F0540FC395F0920B743E
:101900000122788179217A03E6C4540FF309E65461
:101910000FF30908DAF2792178A07A06E6540FF677
:10192000E36670080908DAF4E4C24422792678A54F
:101930007A06C3E3961918DAFA920B792678A57A13
:1019400006E3540FB40F08E6540FB40F108008E6F6
:10195000540FB40F0B80061819DAE680CB740122FD
:10196000C3E396B40902801214600FC3E3F5F0E6F6
:1019700095F0B4090280031470E3E9B42104E4D2C1
:1019800044221918E366540F60F080D112190270D6
:101990001F30441C202E1AC2AF751850858319853C
:1019A000821A120A3F7548B4757700D240D243E4D8
:1019B0002204227408F9747CF8752F0075308C7538
:1019C00031C01204760218CA7408F9747CF8752FB5
:1019D0000075308C7531C012047612198C22740592
:1019E000F9747CF8752F0075308C7531C0120420A5
:1019F000227403F97481F8752F0075308C7531C528
:101A000012042022C082C083E5822420F582E5836F
:101A1000347DF5837401F9743BF8752F00858330AC
:101A2000858231120476D083D082C082C083E58261
:101A300075F008A42420F582500205F0A8F0E58393
:101A400075F008A4282400F5837408F9747CF875EF
:101A50002F00858330858231120476D083D08212A4
:101A60003CF322C082C083E58275F008A42420F5EF
:101A700082500205F0A8F0E58375F008A428240040
:101A8000F5837408F97494F8752F00858330858286
:101A900031120476D083D08222C082C083E5827561
:101AA000F008A42420F582500205F0A8F0E5837523
:101AB000F008A4282400F5837406F9747CF8752FC7
:101AC00000858330858231120476D083D0822274DF
:101AD00005F9747CF8752F007530007531201204FB
:101AE000760218CA900000121A041218CA22300C8A
:101AF000F3751B00751C0075629F75630FE5622509
:101B00001BC2E0F582E563351CF583C082C083E526
:101B1000822400F582E583341BF5837402F9747C1A
:101B2000F8752F01858330858231120476787C86A2
:101B300083088682121A041218CA7005D0F0D0F0F9
:101B400022D083D082C3E58313F583E58213F58227
:101B5000200B14E58245836022E58224FFF562E5CF
:101B60008334FFF5638007A385821B85831CC3E54F
:101B700062951BE563951C40028082740122300C43
:101B8000397410F9747CF8752F017530CE753120D9
:101B90001204767894797C75F00AE7B4FF02801A13
:101BA000B43C120809D5F0F2900FE878C6E2F53B94
:101BB0007854F2E42266540F60E974012290000028
:101BC000121A0412198C2278A0E6540FB40F0302E3
:101BD0001C61200C0280E6751B00751C0075629F5D
:101BE00075630FE562251BC2E0F582E563351CF5E0
:101BF00083C082C083E5822400F582E583343BF50F
:101C0000837402F9747CF8752F01858330858231E5
:101C1000120476787C8683088682121A0412198C44
:101C20007005D0F0D0F022D083D082C3E58313F5C5
:101C300083E58213F582200B14E58245836022E55B
:101C40008224FFF562E58334FFF5638007A3858274
:101C50001B85831CC3E562951BE563951C400280D0
:101C60008274012278947A0579A8E6540FC4F5F0BD
:101C700008E6540F45F0F70809DAEF2275F01E1256
:101C80008696D5F0FA1200E475F00F128696D5F01C
:101C9000FA1200E475F00F128696D5F0FA1200E4FD
:101CA00022120094B2B575F00F128696D5F0FA3074
:101CB000B7EF22D218D2A3C251C2A2D254D2A1C22B
:101CC00053D2A4C252121CA1121C7C121F6D1257B7
:101CD0002B126780120D7E120640C2A3C251C2A20F
:101CE000C254C2A1C253D2A4C252125EF64005C26F
:101CF000AF026466120094B2B575F00F128696D5E5
:101D0000F0FA80E6C2A3C251C2A2C254C2A1C25319
:101D1000D2B775F002128696D5F0FA20B744125E5B
:101D2000F65002808ED218D2A3C251C2A2D254D28F
:101D3000A1C253D2A4C252121CA1D2181257714090
:101D40001CC2A3C251C2A2C254C2A1C253D2A4C2D5
:101D500052121E9612572B120D7E120640C2AF026F
:101D60006466125ED1C01D120949D0F0703BC3E514
:101D70001D95F078ACF2121E301215346019D2188D
:101D8000900000121A04121E9612572B120D7E128A
:101D90000640B2B5121E3012130EE57654087008D4
:101DA00012675D5003121DEB22D2A3C251D2A2C210
:101DB00054C2A1C253D2A4C252C218754AFAC2A0D8
:101DC00075F0C8128696D5F0FA125ECCD2A075F0E6
:101DD000C8128696D5F0FA125ED11232B0D2B7127E
:101DE00086AE20B7C4021D1E020000D2B71286AE16
:101DF00030B7F5D2A3C251D2A2C254C2A1C253D2AB
:101E0000A4C252C218754AFAC2A075F0141286967E
:101E1000D5F0FA125ECCD2A075F014128696D5F0E9
:101E2000FA125ED11259D61232B012675D40BC224E
:101E30001215731216261216C4A2E49272A2E5922B
:101E400073A2E69274A2E792751216ED121747126A
:101E500017ED12186D12175A7401F974B5F8752F31
:101E6000017530CE75313012045178B5E2B4FF02FD
:101E7000E4F27401F974B6F8752F017530CE75313E
:101E80003112045178B6E2B4FF02E4F21218B7122C
:101E9000148512170022D218C2A3C251C2A2C25482
:101EA000C2A1C253D2A4C252C01EC01F787C9000EF
:101EB000007A08E6F008A3DAFA121F6D126780783C
:101EC0007C9000007A08E0F608A3DAFA900000128D
:101ED000569A1219DE1219F1D01FD01E1218A42220
:101EE000751E30751F30D21EC21FC220C201C22B08
:101EF000C22CC22DC216C22FC22ED230C231C23263
:101F0000C234C235C236C238C239C23AC23BC23C00
:101F10007573007574007575007576087870742295
:101F2000F2087400F278727406F2087400F2C27259
:101F3000C273C274C275784F7404F278527409F295
:101F400078567401F278577402F278587404F27873
:101F5000597404F2753807753900753A00740178C0
:101F60005EF2785FF2E408F208F2C20C221209EE87
:101F7000121EE01218A412154C121599C2E0A2729A
:101F800092E4A27392E5A27492E6A27592E7121609
:101F9000AE1216DA1217341217A412183612177F5F
:101FA0001214DD121502125F5022305604C2568000
:101FB0000975F00C20B205D5F0FAD322C322E8C08F
:101FC000E0E9C0E0EAC0E0200637200834121FAA8A
:101FD0005025755000785FE2600C75F0031286960C
:101FE000D5F0FA1222EC785EE2600C75F0031286EE
:101FF00096D5F0FA122451D0E0FAD0E0F9D0E0F80A
:102000002220092220071F3060EDC082C083E56ACC
:102010007008126907400312203D12143E1268D75F
:10202000D083D08280D13060CEC082C083E56A7018
:10203000031220931269E0D083D08280BA30050C5D
:10204000300609D25BC25A785E0220553008F4D2BD
:102050005AC25B785FE2B40F028013B41007123EDD
:10206000A2D24C802D75F00384E5F0B40007123F36
:1020700085D24C801DB40107123E10D24B8013B4A0
:102080000210123D87400B784DE583F208E582F29D
:10209000D24D2230050C300709D25BC25A785E025D
:1020A00020AB3009F4D25AC25B785FE275F003844A
:1020B000E5F0B400091241384020D24C801CB40134
:1020C000091241604014D24B8010124163400B78DA
:1020D0004DE583F208E582F2D24D22D24E8008C24D
:1020E0004E12214D753C00C217D256754AFA744003
:1020F000301802740CF547C24CC23FE547603912F4
:102100001FBE204C3375F003128696D5F0FA1202EA
:102110007A201803201718303FE1204E1B754760C6
:10212000121262B40B0D75F008128696D5F0FAD231
:102130004C800512214080C3C24BD2AF754AFA22AF
:10214000533C07F8E53C24A0C8F6053C2278A0756E
:10215000F00874FFF608D5F0FB22304B09201D0370
:10216000D21D22C24B22C21D22D24E8004D256C2A0
:102170004EC217754AFAD21C7440301802740CF51E
:102180004712214D753C00C24CC24BC23FC24DC2EA
:102190004F12027A20180320172D121FBE204C293F
:1021A000204B26204D23303F2D785EE27004C23F45
:1021B0008024204E14754760121262B40B1275F021
:1021C00008128696D5F0FAD24C757703754AFA2232
:1021D000757703122140E54760F2304FFD80B0B4BF
:1021E0000207204C07C24BC24D02226DC082C08341
:1021F00090EA60E53C606324FB405F78A0E6540F02
:10220000758300F582D53C02805075F00AA4F582F2
:1022100075830008E6540F2582F582D53C02803A8A
:10222000E58275F00AA4F58285F08308E62582F53B
:102230008250020583D53C028020E58275F00AA415
:10224000F582C0F0E58375F00AA4D0F025F0F5839F
:1022500008E62582F58250020583784DE583F20871
:10226000E582F2C24CC24BD24DD083D08222C289C9
:10227000C28BD293C2B422C0F075F0FAD5F0FD75CE
:10228000F064D5F0FDD0F0221222771222771222CC
:102290007712227712227712227722D293C2B47554
:1022A000F0051286AE20B2061286AE30B203D5F02B
:1022B000F11286AE22C0F075F008A2E7B392B4C264
:1022C00093122277C2B4D293122277C0E0E430B2E4
:1022D00001040030B201040030B20104D36003D520
:1022E000E001C3D0E033D5F0D1D0F022D293C2B414
:1022F000D2B2122277C293122288D293122288205D
:102300001803305B1C788C7601087480F608A2A351
:10231000B392E4F6749008F608F608F608F602237D
:1023200061788C7603087680087480A25192E5A2C9
:10233000A3B392E4201808A25492E1A22892E0F6F6
:10234000087480201812205B0FE55054074480A2C7
:102350005392E5A2A1B392E4F6087480F608F60859
:10236000F675F007788C7E007F00E62EFEE61222DE
:10237000B5F62FFF08D5F0F2EED3331222B5F8EF01
:10238000D333687066788CB6FF61055EE55E24FE27
:102390005016755E02201A10D21AC2AF7518C07599
:1023A0001900751A03120A3F201808785FE26003CB
:1023B000305B0302244D7892E620E35B20E24B2061
:1023C000E127788DE6B6002108B6420908E6D25A20
:1023D0001228AB8078B6551108B6000D08794DE685
:1023E000F30809E6F3D24DD25A8062E55E6019D552
:1023F0005E16301A13C21AC2AF7518C0751900756F
:102400001A04120A3F7578038043788D863C08D2FF
:102410004C79A07A04800B788DD24B756B0579943A
:102420007A05D25A75F00FE6C4540FF755F0F5F05F
:1024300009E6540FF755F0F5F00908DAEAE5F0B4CB
:102440000F051977EEC24B785FE21221DF12229B53
:1024500022D293C2B4D2B2122277C293122288D26D
:102460009312228820181F305A23788C7611087412
:1024700080F608A2A3B392E4F6749008F608F60872
:10248000F608F60224D6788C7615022491788C769C
:1024900013087680087480A25192E5A2A3B392E457
:1024A000205A14A25292E1A2A4B392E0201808A2EA
:1024B0005492E1A22892E0F6087480205A0FE55069
:1024C00054074480A25392E5A2A1B392E4F60874A3
:1024D00080F608F608F675F007788C7E007F00E637
:1024E0002EFEE61222B5F62FFF08D5F0F2EED3331A
:1024F0001222B5F8EFD333687064788CB6FF5F05AD
:102500005DE55D24FE5016755D02201B10D21BC2D6
:10251000AF7518C0751900751A05120A3F785EE28A
:102520006003305A030225CB7892E620E36720E26D
:102530005720E14A788DE6B6002208B6420A08E63E
:10254000D25B1228AB0225CBB6551108B6000D0898
:10255000794DE6F30809E6F3D24DD25B806DE55D77
:102560006019D55D16301B13C21BC2AF7518C0753C
:102570001900751A06120A3F7578030225CBD25B43
:10258000788D863FD23F8043788D863C08D24C7947
:10259000A07A04800B788DD24B756B0579947A05FF
:1025A000D25B75F00FE6C4540FF755F0F5F009E66D
:1025B000540FF755F0F5F00908DAEAE5F0B40F0525
:1025C0001977EEC24B785EE21221DF12229B22784D
:1025D0005FE2601024FD400C75F003128696D5F082
:1025E000FA1222EC22785EE2601024FD400C75F0B5
:1025F00003128696D5F0FA12245122C0E0305A0E0A
:10260000C2AF7518B0751900751A00120A3FD0E0F4
:1026100022D293C2B4D2B2122277C293122288D2AB
:1026200093122288788CE56F540FC44407F608E5AE
:102630006E23A2E392E5A2E292E3542AD2E7F608DF
:10264000E56EA2E392E1A2E492E3542AD2E7F6080F
:10265000E56EA2E692E1A2E792E3540AD2E7F674AD
:102660008008F608F608F675F007788C7E007F0083
:10267000E62EFEE61222B5F62FFF08D5F0F2EED3D5
:10268000331222B5F8EFD33368700B788CB6FF069F
:1026900012229BC3800412229BD322756F08787488
:1026A000E2F56E12261174004005122775800312A0
:1026B000279D756F097875E2F56E12261174014039
:1026C00005122775800312279D2222E5735420608E
:1026D000F9756F04756EFF122611740250041227EB
:1026E0009D22122775788F7948E6F30809E6F308EA
:1026F000794AE6F30809E6F3788DE6A2E092E2541F
:1027000014F5F008E623A2E592E0540345F0F5F055
:10271000784CE265F0C0E0E5F0F2D0E030E221C0B4
:10272000E0C0F0E5F075F04930E20375F04AC2AF61
:102730007518C075190085F01A120A3FD0F0D0E064
:1027400054037003022774E5F05403B4030575F0D5
:10275000488013B4020575F047800BB4000575F08E
:102760004B800375F04CC2AF7518C075190085F029
:102770001A120A3F22F5F02442F8E2B4020522744C
:1027800002F22250FA7402F2E5F02432F5F0C2AF00
:102790007518C075190085F01A120A3F22F5F02449
:1027A00042F8E2601CD5E018F2E5F0243CF5F0C2F6
:1027B000AF7518C075190085F01A120A3F757803B5
:1027C000F222D293C2B4D2B2122277C293122288DA
:1027D000D293122288788CE56F540FC44403F60814
:1027E0007680087480A25192E5A2A3B392E4A25429
:1027F00092E1A22892E0F6087480A25392E5A2A189
:10280000B392E4F6087480F608F608F675F00778D7
:102810008C7E007F00E62EFEE61222B5F62FFF0822
:10282000D5F0F2EED3331222B5F8EFD333687071DE
:10283000788CB6FF6C7892E620E33020E22020E12D
:1028400060788DE6B6005A08B6551108B6005208F1
:10285000794DE6F30809E6F3D24D804A8043788D3E
:10286000863C08D24C79A07A04800B788DD24B75C7
:102870006B0579947A0575F00FE6C4540FF755F09F
:10288000F5F009E6540FF755F0F5F00908DAEAE536
:10289000F0B40F051977EEC24B7865E21221DF80A4
:1028A0000512229BD32212229BC322B4FF17D267A8
:1028B0007569051225FBC2AF7518C0751900751A28
:1028C00007120A3F22B4BC030228DEB4BD0302296A
:1028D00010B4BE03022942B4BF0302297422205A55
:1028E000147408F9747CF8752F017530CE75314079
:1028F00012047680127408F9747CF8752F01753013
:10290000CE75314812047674117884F61229A62205
:10291000205A147408F9747CF8752F017530CE753F
:10292000315012047680127408F9747CF8752F0106
:102930007530CE75315812047674127884F61229E7
:10294000A622205A147408F9747CF8752F0175308A
:10295000CE75316012047680127408F9747CF875B3
:102960002F017530CE75316812047674137884F6B1
:102970001229A622205A147408F9747CF8752F01C4
:102980007530CE75317012047680127408F9747C3B
:10299000F8752F017530CE7531781204767414787D
:1029A00084F61229A622787DE61201584004741E8E
:1029B000D322787EE61201A8400C741FD322125C49
:1029C000761200D7C322787CE660F9B4FF08D2679C
:1029D000756905022C1DB402122038031225FB78FC
:1029E00084E6127300400280DB80D3B4090CC0E09F
:1029F0007404126E2BD0E0022C1DB43808787FE6E8
:102A0000122C3080BFB43908787FE6122C3A80B49B
:102A1000B43A27306B221225FB78B6E278B7F27809
:102A20008486F0E5F0543F4480C2AF7518C0751934
:102A300009F51A120A3F8086808AB43B24306BF86D
:102A40001225FBE478B7F2788486F0E5F0543F4431
:102A500040C2AF7518C0751909F51A120A3F02294C
:102A6000BEB43C0C1225FB7884E61274870229BEA2
:102A7000B43D391225FB203E18D23EC270C2AF755C
:102A8000187075190F751AE9120A3F757903022932
:102A9000BEC23ED270C2AF75186075190F751AE9C3
:102AA000120A3F75790312424A0229BEB43E13E569
:102AB000735410600A1225FBE4122C3F0229BE0257
:102AC00029C4B43F14E5735410600B1225FB74FF46
:102AD000122C3F0229BE0229C4B4400C1225FB78F7
:102AE00084E612737C0229BEB4410C1225FB788463
:102AF000E61273DF0229BEB4420C1225FB7884E68D
:102B00001273BE0229BEB4430C1225FB7884E61270
:102B1000739D0229BEB4440E7400126E2B7884E6B5
:102B20001286E20229BEB4450E7400126E577884F4
:102B3000E61286F30229BEB446097400126E744090
:102B4000E880D5B4470E7402126E2B7884E61287A3
:102B5000040229BEB4480E7402126E577884E6123D
:102B600087150229BEB449097402126E7440E880C8
:102B7000D5B44A0E7403126E2B7884E612872602AF
:102B800029BEB44B0E7403126E577884E612873751
:102B90000229BEB44C097403126E7440E880D5B4A7
:102BA0004D1A1287487884E6543F4480C2AFF51A24
:102BB00075190B7518C0120A3F0229BEB44E0C30AD
:102BC0003E061225FB022A910229BEB44F09203E7F
:102BD000F71225FB022A79B4540B7400788446124C
:102BE00086290229BEB45504744080F0B45604749A
:102BF0008080E9B4570474C080E2B4580B74007844
:102C000084461286130229BEB45904744080F0B47D
:102C10005A04748080E9B45B0474C080E21225FB1E
:102C2000C2AF7518C0751907F51A120A3F0229C4F8
:102C30001274007884E678B2F22212740A80F47872
:102C400074F208F212269B7884E6543F44C0C2AF67
:102C5000F51A75190B7518C0020A3F700575601ECC
:102C60008002D21522C298C299322018F830991EDB
:102C7000C299204A057534008014C0F0C0E0C0D06D
:102C800075D010E534122FA8D0D0D0E0D0F0209825
:102C90000132C298204AFAC0F0C0E0C0D075D0100E
:102CA000304905C249754000E54424FE400375449F
:102CB00002E54020E72520E61FE540540723245E77
:102CC000C0E07400342EC0E0E5992205402543F5AC
:102CD00043D0D0D0E0D0F032023324543F23232419
:102CE0005FC0E07400342DC0E0E59922155F80DB01
:102CF00080D9D55FFBB54312D213E8C0E078AA743F
:102D0000FAF2D0E0F875400080C7022E6EB462FA85
:102D100080B980B7B42AF380B2F55F24C6E55F407E
:102D2000E924F5E55F50E3055F80A0781AF2155FAE
:102D30008099781BF2155F8092781CF2155F808B6A
:102D4000781DF2155F8084781EF2155F022CCB7817
:102D50001FF2155F022CCB7820F2155F022CCB02FC
:102D60002E9200022D0D00022D1200022D140002E1
:102D70002D1900022CEC00022CEC00022CEC0002BD
:102D80002CEC00022D2B00022D3200022D39000206
:102D90002D4000022D4700022D4F00022D5700024A
:102DA0002CF200022CF200022CF200022CF20002A3
:102DB0002CF200022CF200022CF200022CF2000293
:102DC0002CF200022CF200022CF200022CF2000283
:102DD0002CF200022CF200022CF200022CF2000273
:102DE0002CF200022CF200022CF200022CF2000263
:102DF0002CF200022CF200022CF200022CF2000253
:102E00002CF200022CF200022CF200022CF2000242
:102E10002CF200022CF200022CF200022CF2000232
:102E20002CF200022CF200022CF200022CF2000222
:102E30002CF200022CF200022CF200022CF2000212
:102E40002CF200022CF200022CF200022CF2000202
:102E50002CF200022CF200022CF200022E92800EC4
:102E60008039803D80418044804780548052B4093D
:102E700009754300754000022CCBB421097543004D
:102E8000754040022CCBB442097543007540800266
:102E90002CCB754300754000022CD1B51ED0022CFE
:102EA000CBB51FCA022CCBF541022CCBF542022C2C
:102EB000CBB543BA754420122EC2754000022CD106
:102EC00080D08541361262BBD24AE536B446030251
:102ED0004A69B447041262D122B4500E85423512B9
:102EE0006296C2ACC24A756D0722B4531285423550
:102EF000E542700A126296C2ACC24A756D0222B4F3
:102F0000540E854235126296C2ACC24A756D0122DA
:102F1000B4550E854235126296C2ACC24A756D0335
:102F200022B4560E854235126296C2ACC24A756D05
:102F30000422B4570E854235126296C2ACC24A755D
:102F40006D0522B4580E854235126296C2ACC24A53
:102F5000756D0622B44E3D854235E542B4000B1234
:102F60006296C2ACC24A756D0822B4010B12629619
:102F7000C2ACC24A756D0922B4020B126296C2AC91
:102F8000C24A756D0E22B4030B126296C2ACC24ADD
:102F9000756D0F2224BF24E6400485423522C24AC3
:102FA00022C5372537C53722E53424F0400EE534F5
:102FB0002324C7C0E07400342FC0E022759906C2F4
:102FC0004A753400D2B622802F8034803680388013
:102FD00039803E804680488051804F804D804B80B4
:102FE000468050800E02306F753403F599122FA180
:102FF000053422E53502301D753700740380ECE599
:103000001E80E8E51F80E40230CBE53775340F8081
:10301000DA120A7D122C5B883580D0E53580C9E54F
:1030200035A23E92E080C1753403A8350535E676B9
:10303000FF80B8E535C313603214700BA22592E00F
:10304000B392E1440480D614700BA22692E0B392AE
:10305000E1440880C8147008A22792E0440C80BDA7
:10306000147008A20392E0440C80B274FC80AEE5B8
:103070003514702574083057123058044406809D6A
:103080003059044403809644078092A25892E0A2EB
:103090005992E1A22892E280841470157410A2253E
:1030A00092E0A22692E1A22792E2A20392E30230EA
:1030B0001D14700D7418A21A92E0A21B92E1023046
:1030C0001D14700302301DE402301DE536B44106C4
:1030D000753404022FEBB44212E53560033015035A
:1030E000120A9575601E7442022FE8B4440280F8FB
:1030F000B44B02800302318CE53554F8B4083AE54C
:10310000355407700A741912737CE5360231C3B462
:10311000010A741912739DE5360231C3B4020A74B0
:10312000191273BEE5360231C3B4030A741912735F
:10313000DFE5360231C3022FBCB42003022FBCB43A
:103140002826E53520E008303E0B12424A80062052
:103150003E031264EEE535A2E0923E75680150032D
:10316000756802E536022FE8B4300CE53554F812E4
:103170006E2BE536022FE8B4380CE53554F8126EA4
:1031800057E536022FE8022FBC022FBCB4430FB51F
:1031900035037545037534077535A8022FEBB44A1E
:1031A00028E535702120591E2057087419125ED663
:1031B000125EC4C2AF75181075190F751AF0120A95
:1031C0003FE536022FE8022FBCB4450675340602EF
:1031D0002FEBB4510675340C022FEBB44D0EE535D0
:1031E00012718BE5365002B2E70230E8B44C067536
:1031F000340E022FEBB4460280C9B4470280C4B437
:103200004F08C240C241C24280B9B45917E5357077
:1032100013E8C0E078ACE2F535D0E0F874597534C5
:103220000D022FEB022FBCE56DB4000122C2AC12DF
:1032300086C61286C6D299E56DB407061232C1025F
:1032400032A5B401061210CB0232A5B40306121146
:10325000500232A5B40206120FEC0232A5B40406E5
:1032600012102E0232A5B405061202DC0232A5B4F9
:1032700006061211980232A5B40806125D640232E5
:10328000A5B40906125CE80232A5B40E06125DF17F
:103290000232A5B40F06125E380232A5B41006122F
:1032A00033CD0232A5C24AD2B6126296756D0022A3
:1032B000E56DB4000122C24AD2B6126296756D0065
:1032C0002212608DC2B675370074031249E9E51EFB
:1032D0001249E9E51F1249E974501249E9747D1257
:1032E00049E9900000E535600F9003E8146009900B
:1032F00007D0146003900BB87E7D7F0875F000C086
:10330000F012608DB40203D38001C3D0E033F5F036
:10331000A3DFEC1249E9DEE2E5371249E93099FD15
:1033200022022E9220E5FA20E4F7540F23243AC01B
:10333000E074003433C0E0E5992280E5801F8023EB
:103340008027802A803B80398037803580338031E8
:10335000802F802D802B80298043022E6EB51EFA8F
:10336000022CCBB51FF4022CCBF541022CCBF5423D
:10337000600924F5E54240E2022CCB75404E022C58
:10338000CBF5F0E54024BBC0E02410F8E5F0F2D026
:10339000E005E06542F8E5F0B800E380DEB543BA49
:1033A000754420754000126296C2ACC24A756D1019
:1033B000022CD1854236753500800EE5424480F5F9
:1033C0003675350174017810F212344622E541B4A5
:1033D000284AE54224FD50E3C082C0837810E2F51C
:1033E0008308E2F58208E2B4030A74191242551206
:1033F00060648022B4020A7419124284125FE3806E
:1034000015B4010A741912428D12603B80087419B8
:10341000124296125FBAD083D0828097B42925E5F4
:103420004224FE5096C082C0837810E2F58308E201
:10343000F58212608D7812F2753503854236D0839D
:10344000D08280858086C2B675370074231249E920
:10345000E51E1249E9E51F1249E9E5361249E9E599
:10346000351249E9E535600E7810E2F5F0E5F01225
:1034700049E908D535F4E5371249E93099FD22E5E7
:1034800061C25E6002D25E85515278CF76FFC27112
:10349000C243204D0C204B1B304C030235BE023A78
:1034A000AE120102784DE2F58308E2F582121A04A9
:1034B000023639120102121C64121AEE6019121B34
:1034C0007E603D1225FBC2AF75182075190F751A65
:1034D000EC120A3F0235031242EAB40206123A0124
:1034E000023AAEB4031AC082C0831200E41220DF95
:1034F000D083D082304C0CE53C600812198C7003EC
:1035000002363975493CD54519C2AF7518C07519D1
:1035100000751A53120A3F754503757700D241753D
:1035200048B4023A99D2677569051225FBC2AF7596
:1035300018C0751900751A07120A3F755004122534
:10354000CF1225E575F06412011E023AAE205A240E
:10355000E575540860CC300C18C0E0C082C083749C
:1035600011120188D083D082D0E0400280B70235AA
:1035700095023595E574548060A8300C18C0E0C001
:1035800082C0837410120188D083D082D0E04002C0
:1035900080930235951274D1401E205915302C03AA
:1035A000203E09900FE9123AD6023AAE123A2B02A7
:1035B0003AAE123A31023AAE123A37023AAE12013C
:1035C00002E53C608878A0E6B40A0302423C121B84
:1035D000C770391242EAB40106123A01023AAEB497
:1035E00003241200E4C082C08312216DD083D082F4
:1035F000304B16C082C083120102121C64D083D0EB
:10360000821218CA7003023639023503785E205BD5
:1036100002785FE2B40F0A123E5AC24CD24B023417
:10362000B6B4100280F11225FBC2AF7518207519CF
:103630000F751AEB120A3F80D0305A30300C19C087
:10364000E0C082C083740C120188D083D082D0E0A5
:10365000400302366C023658756F027860E2786576
:10366000F212144A123FD35003023503305B30305C
:103670000C19C0E0C082C083740D120188D083D0C1
:1036800082D0E0400302369F02368B756F0378616B
:10369000E27865F2121456123FD35003023503123A
:1036A0006496400312226EE53B04700302350375F5
:1036B0004900754503C242C241204302C240C08254
:1036C000C083123C09D083D0825006123A46023A97
:1036D000AEC082C083120656D083D0825006123A02
:1036E00046023AAEE58224CEE58334FF5043123BD6
:1036F00069403E1285465006123A37023AAE023908
:103700003C123A370238CE123A310238CE123A2BF6
:103710000238CE123B72500F123CF330E109302CCC
:1037200024123A2B023AAE12854640F2D271023987
:103730003C1274D140CB2059CE303E09E57654205E
:1037400070D1202CC8305A037854E2305B02E53B3C
:10375000120158500902379F123A250238CE300C18
:10376000F7303BF412412A4036A25A303C01B350A4
:103770002E300C18C0E0C082C0837409120188D0BA
:1037800083D082D0E0400280CF02378CC082C083D9
:103790001260E1D083D0825006123A3C0238CE78D3
:1037A000CE76FFD237300C19C0E0C082C0837414CB
:1037B000120188D083D082D0E040030237C30237A1
:1037C000C1C23712412A500302384FA25A303C017D
:1037D000B3920A5016126137501130370812608DBB
:1037E000B402028006123A130238CE12608DB40081
:1037F00005200A278043B4013A200A1F301650C220
:10380000AF7518C0751900751A09120A3F203706DE
:10381000123A410238CE123B2C8034E576541070B7
:103820000912429F78CF7602802512429F78CE7689
:1038300002801CB402DA200AC3E576541070091223
:10384000429F78CF7601800712429F78CE76013072
:103850000C5C12412A4057300C19C0E0C082C08372
:103860007408120188D083D082D0E040030238AEC1
:10387000023873205E1CA25A925D78D1A68378D25A
:10388000A682123B28C25AC25B1200F8756102027E
:103890003AAE756100E58378D166F5F0E58278D2BD
:1038A0006645F07006123A4B0238CE1241C7123A02
:1038B000D6E57654106006300F031242AAE5735421
:1038C00010600BC082C083123D19D083D082E57690
:1038D0005420600C30710975F0C812011E023AAE16
:1038E000123B725009123CF330E103023AAE1285EA
:1038F0004640F8C2A1D253D2A4C25275500012253C
:10390000CF1225E5121A04C082C08312216DD08324
:10391000D082204D09204B17204C1C023AAE1201D8
:1039200002784DE2B5830D08E2B5820802393C12F7
:1039300018CA6008023A9912198C70F878CF76FF8D
:10394000300C19C0E0C082C0837406120188D08395
:10395000D082D0E04003023A9902395CE573540109
:10396000601FE58245836019305A037854E2305B6A
:1039700002E53B1201585003023981123A19023A0A
:10398000AEA23E92701274E4500F123A1F75F01EF0
:1039900012011E1200C1023AAEB23E1225FB303EA9
:1039A00022C2AF75187085831985821A120A3F7575
:1039B0007903C2A3C251D2A1C253D2A4C25212648B
:1039C000EE8038C2AF75186085831985821A120A95
:1039D0003F757903D2A3C251D2A1C253C2A4C2522D
:1039E00012424AE57654206012E58224CEE5833403
:1039F000FF5005123B6950030237451200D7023AC7
:103A0000AE125C6C023A4E125C6C023A4E125C6C66
:103A1000023A4E125C6C023A4E125C6C023A4E1242
:103A20005C6C023A4E125C6C023A4E125C6C023ACA
:103A30004E125C6C023A4E125C6C8012125C6C800E
:103A40000D125C6C8008125C6C8003125C6C7561FA
:103A50000078D176FF78D276FFD26E1225FBC2AF06
:103A600075182085831985821A120A3F1200C1C277
:103A70006E22E57454087003205A1DE55104601845
:103A800014F5F07855E265F0600EC2AF7518C07598
:103A9000190185511A120A3F22125C6CD26E120073
:103AA000ABC26E75610078D176FF78D276FFC24CDA
:103AB000C24BE552F55178CFE6B4020A741C1242AB
:103AC00084125FE3800BB40108741C12428D1260F3
:103AD0003B78CF76FF22303E0EC2A3C251C2A2C2B3
:103AE00054D2A4C252800CD2A3C251C2A2C254C2A8
:103AF000A4C252A25A920ED20D125C6C741C125EB9
:103B0000D6125EC4E5735440600620A80312856D8A
:103B10001225FB123A72C2AF75181085831985827F
:103B20001A120A3F1200D722125C6C22125C6C75CA
:103B3000F03212011E227408F9747CF8752F017599
:103B400030037531901204767881E60856085604E1
:103B500060141200E41220DF304C09E53C600512CD
:103B6000198C6002C322D32222E582249CE583348F
:103B7000FF22E582249CE58334FF22E5822582F53D
:103B800082E5833583F583E5822582F582E58335F9
:103B900083F583E5822400F582E583345BF5837445
:103BA00004F97400F8752F01858330858231120481
:103BB00051227881E654C0F5837882E630E402240D
:103BC0000A2323543C4583F5837881E6C454037566
:103BD000F00AA4F5F0E6540F25F0030303F5F053C3
:103BE000F0E085F08254034583F5837880E6C45481
:103BF0000375F00AA4F5F0E6540F25F04582F5822E
:103C000022C39582E5F095832212412A5003023C9B
:103C100091123B7B7800E2B4FF03023C911267E40F
:103C2000123BB2787CA68308A6827800E2F583086E
:103C3000E2F58208E2F5F008E2123C01502B780030
:103C4000E2F58308E2F582787C86F008E6123C0112
:103C500050417802E2F58308E2F582787C86F0082C
:103C6000E6123C01402D023C917800E2F58308E227
:103C7000F582787C86F008E6123C0140167802E274
:103C8000F58308E2F582787C86F008E6123C015064
:103C900002C322D322C3E58233F582E58333F58361
:103CA000E5822400F582E583349AF5837402F97481
:103CB00053F8752F0185833085823112045122C358
:103CC000E58233F582E58333F583E5822400F582CE
:103CD000E583349AF5837402F97453F8752F0185DE
:103CE00083308582311203EF2278537400F208E4A6
:103CF000F2801E300CF3C082C083123C95D083D07A
:103D000082E5822418E58334FC40067853E24402BD
:103D1000F27854E2F5F018E222E5822400F582E51B
:103D20008334BAF5837401F9747CF8752F018583A7
:103D300030858231120476787CE660422323C0E02D
:103D40005403F5F0D0E054FC2400F582E5F034CAC9
:103D5000F5837404F9747CF8752F018583308582AE
:103D600031120476787CE60886F07874F208E5F083
:103D7000F275F002128696D5F0FA12269B2274FF95
:103D80007874F208F280EAE56CB4220575F00480DC
:103D900013B42A0575F006800BB4420575F00C804B
:103DA0000375F0027830E2540F704F08D5F0F7E257
:103DB000540F75F00AA4F58275830008E2540F25AC
:103DC00082F582E58275F00AA4F58285F08308E227
:103DD0002582F58250020583E58275F00AA4F582FA
:103DE000C0F0E58375F00AA4D0F025F0F58308E271
:103DF0002582F58250020583C322D3227830E26007
:103E00000BF5F008E2240A4005D5F0F7C322D322CF
:103E1000783079947700097700097700097700E511
:103E20006CB4220A756B04799675F0088024B42A64
:103E30000A756B05799475F00A8017B4420C756B9E
:103E400005799475F00A78368008756B0379987552
:103E5000F006E2F70809D5F0F922C082C083789411
:103E60009002E475F00AE0F608A3D5F0F99002EEAE
:103E7000E0F56BD083D08222C082C0837894900218
:103E8000E475F00AE6F008A3D5F0F9E56B9002EED0
:103E9000F0D083D08222123E101218CA22D083D0D2
:103EA0008222123E10123E7812214DC082C08375CC
:103EB0003C017830E2540F70E408E2540F70DE08E1
:103EC000E2540FC4F5F008E2540F45F0F58308E220
:103ED000540FC4F5F008E2540F45F0F582C264783F
:103EE000A07900C3E5829410F582E5839427F583D9
:103EF00040030980EEE5822410F582E5833427F53E
:103F000083E96004D264F6087900C3E58294E8F599
:103F100082E5839403F58340030980EEE58224E87B
:103F2000F582E5833403F583E92064046004D264F8
:103F3000F6087900C3E5829464F582E5839400F580
:103F40008340030980EEE5822464F582E583340032
:103F5000F583E92064046004D264F608E58275F014
:103F60000A842064026002F608E5F0F6E82461F5B0
:103F70003CD083D0822279A077000975F00577FFC5
:103F800009D5F0FA22123E10123E78123F7675F0F3
:103F900008E56CB4220478308013B42A04783280A7
:103FA0000CB4420478388005783075F006753C060C
:103FB000E2540F700608D5F0F7800979A0E2F708FF
:103FC00009D5F0F922123F8512198C22123EA21255
:103FD000198C227865E2700302408824FD4038C0C5
:103FE00082C0831200E41240E4D083D082204D16B8
:103FF000204C0B304B361218CA703102408812190F
:104000008C7029024088784DE2B5832008E2B582A1
:104010001B658270178071E224E24070C082C08309
:104020001200E41269A9D083D082500302408A783A
:1040300065E2B40F0C123FC5604E123E9660498097
:10404000EBB41007123FCC603F80E175F00384E5CC
:10405000F0B40007123FC570D3802DB40107123EA3
:104060009670C98023B4021EC082C083123D87E5CA
:10407000828583F0D083D08240B2658270AEE5F055
:10408000658370A8800280A4C322D322C082C0832B
:104090001200E41269FFD083D0825002D3227865E7
:1040A000E275F00384E5F0B4000A12413812198C6D
:1040B00070EA802CB4010A1241601218CA70DD80C7
:1040C0001FB4021EC082C083124163E5828583F063
:1040D000D083D08240C6658270C2E5F0658370BC33
:1040E000C32280B8754732D256304F09C24FC06FD5
:1040F00012027AD06FE547D36018C24DC24CC24B52
:10410000121FAA50E41227C2204D06204C03304B48
:10411000D8C3C0D0A86F7405B802027404D0D040D0
:1041200005122775800312279D22E582B4E807E572
:1041300083B40F02D322C322123DFC5002D3227853
:1041400030E260F9F5F008753C06E2540F7006089D
:10415000D5F0F7800979A0E2F70809D5F0F9C32274
:10416000026B21123DFC5004D322C3227830E208B6
:1041700060F6B40108E2F58275830080EDB40212A6
:10418000E275F00AA4F58208E22582F582758300C3
:1041900080D8B40320E275F00AA4F58208E22582F3
:1041A00075F00AA4F58285F08308E22582F5825035
:1041B000B9058380B5B404057831023DAFC39404DA
:1041C000F5F07831023DA6B25AB25B755007122560
:1041D000CF1225E5B25BB25AC2AF7518C07519008F
:1041E000751A0C120A3F305D0EC2AF7518B0751902
:1041F00000751A00120A3F123A72C082C08378D149
:10420000868378D28682C2AF75181085831985821D
:104210001A120A3FD083D08222E53CB4031C78A056
:10422000E6B40A1608E624F6401008E624F6400A2A
:1042300018E675F00AA40826C322D32212421950A8
:10424000030235CE78B0F20243451264EE1287487D
:10425000C240C2432230162B543F44C0C082C083A8
:10426000C0E0C2AF7518E085831985821A120A3F33
:10427000D0E0C2AFF51A75190E7518C0120A3FD0FA
:1042800083D082223016FC543F448080CF3016F316
:10429000543F444080C63016EA543F440080BD7805
:1042A000ADE582F278AEE583F22278CEE6B401186D
:1042B000C082C08378ADE2F58278AEE2F583741CEB
:1042C00012428D12603B8019B4021AC082C08378FA
:1042D000ADE2F58278AEE2F583741C124284125F7F
:1042E000E3D083D08278CE76FF22205A0AE4A272ED
:1042F00092E0A27392E122E4A27492E0A27592E1AC
:1043000022439C43BE43FA4370437043704370445E
:1043100026443444424450445E449944CD44D544F8
:10432000E744F54533458745AC45C345E646044675
:1043300022462E464C466A4676469446B246BE46CD
:10434000D9495D499378B0E224DE402412487B408D
:104350001378B0E225E00490430193C0E0E225E049
:1043600093C0E0220249351249341200D7023AAE16
:10437000740A024935D2A1C253C2A4D2521249339F
:104380001200E412216D204C02D322E53CB402F964
:1043900078A0E624F640F208E624F622124932120A
:1043A0004375401578A0E62430F51E08E62430F564
:1043B0001F1218A412572B80AE74200249351249DF
:1043C0003212481A402F1267E478A0E6C40846F576
:1043D000F078A4E65403030345F07881F678A2E66A
:1043E000C40846F5F078A5E6C42345F07882F612B5
:1043F0006796024367741E0249351249321247CB51
:10440000401F1267E478A0E6C408467880F678A2D8
:10441000E6C40846787FF6E4787EF6126796024393
:1044200067741F024935124932124914741B127302
:104430007C024367124932124914741B12739D02A5
:104440004367124932124914741B1273DF02436727
:10445000124932124914741B1273BE024367124987
:1044600032128546402E1249141264EE128748C259
:1044700040C243C23ED270784DE2F58308E2F58235
:10448000C2AF75186085831985821A120A3F757943
:1044900003024367741602493512493212854640B9
:1044A000F31274E440EEC2701249141264EED23E6C
:1044B000784DE2F58308E2F582C2AF751870858306
:1044C0001985821A120A3F7579030243671249322D
:1044D000203E8B80C412493212491475F0C81286EE
:1044E00096D5F0FA026466124932124914741B120E
:1044F000748702436712493220170D124793402EEA
:10450000124948402978B1F278B1E2F551F55212DA
:104510004914C2AF7518C085511A751903301703B5
:10452000751902120A3F0243677419024935741A59
:1045300002493512493220170D12479340F01249B3
:104540004840EB78B1F278B1E2F551124914C2AFAC
:104550007518C085511A751906301703751905129B
:104560000A3F1259D6125A0D123B68D2A2C254C247
:10457000A1D2531200E412216D7418204B06204C76
:1045800003304DAC023492124932306B2F78B6E2D0
:1045900078B7F2124914741B543F4480C2AF7518A7
:1045A000C0751909F51A120A3F02436712493230E1
:1045B0006B0A124793500A741C024935741D024954
:1045C0003570CD124932306BF3E478B7F2124914EA
:1045D000741B543F4440C2AF7518C0751909F51AD1
:1045E000120A3F0243671249327400126E2B741B89
:1045F000543F4400C2AF7518C075190AF51A120A63
:104600003F0243671249327400126E57741B543FC5
:104610004480C2AF7518C075190AF51A120A3F0214
:1046200043671249327400126E7440DB80BB12493A
:10463000327402126E2B741B543F4400C2AF7518C3
:10464000C075190CF51A120A3F02436712493274F9
:1046500002126E57741B543F4440C2AF7518C075A8
:10466000190CF51A120A3F024367124932740212FA
:104670006E7440DB80BB1249327403126E2B741BC4
:10468000543F4480C2AF7518C075190CF51A120A50
:104690003F0243671249327403126E57741B543F32
:1046A00044C0C2AF7518C075190CF51A120A3F0242
:1046B00043671249327403126E7440DB80BB74048A
:1046C000126E2B741B543F4440C2AF7518C075194D
:1046D0000BF51A120A3F024367128748741B543FB6
:1046E0004480C2AF7518C075190BF51A120A3F0243
:1046F0004367C2A1D253C2A4D252123B681200E453
:1047000012216D204D09204B1F204C510247267865
:104710004DE2F58308E2F582120102300C06123CEC
:10472000F320E202C322D322121AEE70F91242EAF7
:10473000B4020280F1B4031AC082C0831200E412F2
:1047400020DFD083D082304CDDE53C60D912198C5B
:1047500070D4784DE583F208E582F280BB121BC766
:1047600070C41242EAB4010280BCB40324C082C007
:10477000831200E412216DD083D082304BA8C08216
:10478000C083120102121C64D083D0821218CA7036
:104790009580BFD2A1C253C2A4D252124933120093
:1047A000E412216D204C02D322E53C60FA24FC4047
:1047B000F6A93C78A07A00EA75F00AA42640E8C57C
:1047C000F070E4AAF008D9EFEAC322D2A1C253C222
:1047D000A4D2521249331200E412216D204C02D3AC
:1047E00022E53CB404F9F5F078A0E624F640F008A0
:1047F000D5F0F778A0E675F00AA4082624E8402E44
:1048000078A2E675F00AA4082624C4402122E0E23A
:10481000E0E1E0E1E0E0E1E0E1E0D2A1C253C2A4E6
:10482000D2521249331200E412216D204C02D322DD
:10483000E53CB406F9F5F078A0E624F640F008D59A
:10484000F0F778A2E675F00AA4082660E1C0E0243B
:10485000F3D0E040D990480D93F978A0E675F00ABE
:10486000A4082660C9C0E029D0E040C278A4E624AC
:10487000F640BB78A5E624F940B422300C7C784D94
:10488000740FF20874E9F220177C78B0E22400F586
:10489000827583D07401F9747CF8752F018583309B
:1048A000858231120476787CE6120158506278B025
:1048B000E22400F5827583D17401F9747CF8752FB8
:1048C00001858330858231120476787CE61201A856
:1048D000503678B0E22400F5827583CF7401F97404
:1048E0007CF8752F01858330858231120476787CBF
:1048F000E6205A0C20E01530E10C1246F2740D222D
:1049000020E20920E3F4C322740E8006740C8002B6
:10491000740BD32220171A1225FB784DE2F5830879
:10492000E2F582C2AF7518E085831985821A120AF2
:104930003F22222222C0E0125C6C124932D0E012E7
:10494000584F1200AB023AAEC051C082C083F5513D
:104950001258D2D083D082E551D051B322124932BD
:10496000D2A1C253C2A4D2521249331200E412217E
:104970006D204C02D322E53CB401F978A0E654FC4A
:1049800070F2E60303441CC0E0124914D0E0128622
:1049900013C322124932D2A1C253C2A4D252124925
:1049A000331200E412216D204C02D322E53CB40105
:1049B000F978A0E654FC70F2E60303441CC0E01250
:1049C0004914D0E0128629C322C5372537C53722BE
:1049D000E54924E94008D2A3C251D2A2C25430987A
:1049E000EFC298E5991249C9223099FDC299F5990B
:1049F0001249C922C2A3C251C2A2C254C2B675375B
:104A00000074051249E9E51E1249E9E51F1249E95A
:104A1000221286C61286C61286C61249F4E53612DE
:104A200049E9E5371249E93099FD221209AD024AF8
:104A300034120949C0E01249F4E5361249E9D0E0E0
:104A40001249E9E5371249E93099FD221286C6126A
:104A500049F4E5361249E9797CE71249E909DDF9BB
:104A6000E5371249E93099FD22D218754919751AAE
:104A700000128748E538600B54F87007C229A22954
:104A8000B392A5E539600B54F87007C22AA22AB385
:104A900092A6E53A600B54F87007C204A204B392E0
:104AA00080125ED1C28EC28CC2ADC2ABC2ACC2AFEC
:104AB0007581D3904ABEC082C08375D00032D2AF18
:104AC000D28C126296C2ACD299124A11B2B5754913
:104AD00019D298024AFBB40922F5371249D0B51E03
:104AE000271249D0B51F211249D0B4461B1249D014
:104AF000AF371249D06F7010124A11D2B6D2A3C28A
:104B000051D2A2C2541249D0B40ACBF5371249D0BF
:104B1000B51EF51249D0B51FEF1249D0F536B46D68
:104B200003024BABB46E03024BC4B46F03024BFBE6
:104B3000B47003024C48B47103024C5CB4730302BA
:104B40004C6DB47403024C6FB47503024C83B4769D
:104B500003024BF8B47703024C9BB47803024CAFCA
:104B6000B47903024CD0B47A03024CECB46C030267
:104B70004D00B46B03024D22B46A03024D5DB4696B
:104B800003024D79B46803024DD5B46703024DEDBD
:104B9000B46603024E08B46503024ECCB46303024C
:104BA00055D7B46103025642024AFBAF371249D0CF
:104BB0006F70F5124A11D2B675F01E128696D5F0B6
:104BC000FA0264661249D0FD1424E0402B1249D049
:104BD0002400FC7B001249D0FEAF371249D06F7021
:104BE000178EF0EDF9747CF88B2F8C3085F0311234
:104BF0000476124A4C754919024AFB1249D0FD1439
:104C000054E070F41249D02400FC247140EA7B0285
:104C10001249D0FEEDFA787C1249D0F608DAF9AFE5
:104C2000371249D06F70D1C2A3C251C2A2C2548EF2
:104C3000F0EDF9747CF88B2F8C3085F03112042064
:104C4000124A1A75491980B0AF371249D06F70A84F
:104C500012076D124A11754919024AFBAF37124902
:104C6000D06F7009124A31754919024AFB808912C6
:104C700049D0FD1424E040341249D02400FC7B01CB
:104C8000024BD51249D0FD1454E070201249D024B3
:104C900000FC242540167B03024C10AF371249D08C
:104CA0006F7009124A2B754919024AFB024BF879B9
:104CB0001A7D071249D0F309DDFCAF371249D06FD6
:104CC00070EA12585140E5126796124A1A024AFBDE
:104CD000AF371249D06F70D41267E41286C61249FA
:104CE000F4E5361249E91202F8024AFBAF371249DD
:104CF000D06F7066120D7E124A11754919024AFB77
:104D00001249D0FE1249D0FD1249D0FCAF371249EA
:104D1000D06F70461206D34041124A1175491902EC
:104D20004AFB1249D0FE1249D0FDAF371249D06F6D
:104D300070281206A41286C61286C61249F4E536F9
:104D40001249E9EE1249E9ED1249E9EC1249E9E5A7
:104D5000371249E93099FD024AFB024BF8AF37128E
:104D600049D06F70F51286C61286C61249F4E53630
:104D70001249E91211B1024AFBAF371249D06F70E4
:104D8000D912094160027401C0E01209A5600274E1
:104D900002D0F045F070071207B8121502E4C0E027
:104DA0001249F4E5361249E9D0E0C0E01249E9E5DC
:104DB000371249E975F003128696D5F0FA1249F4D4
:104DC000E5361249E9D0E01249E9E5371249E93000
:104DD00099FD024AFB1249D0FD1454E07027124994
:104DE000D02400FC2471401D7B00024C101249D0DD
:104DF000FD1454E0700F1249D02400FC2425400516
:104E00007B01024C10024BF8AF371249D06F70F59E
:104E10001286C61286C61249F4E5361249E97402B2
:104E20001249E9744E1249E974831249E97448122F
:104E300049E974311249E974001249E9748D124943
:104E4000E974201249E974DA1249E974001249E957
:104E5000740F1249E974A01249E974801249E97487
:104E6000001249E974001249E974201249E97400FA
:104E70001249E974001249E974001249E9740012F8
:104E800049E974001249E974001249E974001249B1
:104E9000E974001249E974001249E974001249E901
:104EA00074001249E974001249E974001249E97466
:104EB000001249E974001249E974001249E9E53722
:104EC0001249E93099FD024AFB024BF81249D0F52C
:104ED000831249D0F5822460E58334F040EB12510F
:104EE000581249D0FD1454E070DF780075F020743A
:104EF000FFF208D5F0FB78001249D0F208DDF9AFD7
:104F0000371249D06F70C2124A1175F00512869699
:104F1000D5F0FA124A1A751A01300CAD12518E12E0
:104F20005174125166121A04789479007A0A75F055
:104F30000FE3540FF652F00809DAF643F0F0E5F00B
:104F400004789D79807A051218DD600B124FED50C0
:104F500006751A04024EC9125174125166121A04CF
:104F600078A0790A7A0675F00FE3540FF652F0082C
:104F700009DAF643F0F0E5F00478A579837A0312B4
:104F800018DD600B12508B5006751A06024EC912BE
:104F900051741251D7751A65024AFBC0E0782AE5B0
:104FA00083F208E582F2D0E022C0E0782CE583F2BB
:104FB00008E582F2D0E022C0E0782AE2F58308E238
:104FC000F582D0E022C0E0782CE2F58308E2F58299
:104FD000D0E022E5822400F582E583341BF58322AC
:104FE000E5822400F582E583343BF5832212516685
:104FF000AB83AC82901B00C0837900752F0385833F
:10500000307531009000561203D51204E51203D515
:1050100012052F9000567A80E0A3F5F0E0A36C70A3
:1050200005E5F06B6017DAF0D0830583740024C0C7
:10503000E58334C550C1740512513AD322D083EAB6
:105040002AF5F0E4C395F0F582124F9B789479002D
:105050007A0A75F00FE3540FF652F00809DAF643B6
:10506000F0F0E5F004600C121AF1700A74061251A7
:105070003AD322121AF1E5822582F582E58335833F
:10508000F583124FD3124FA90253DF125166AB833F
:10509000AC82903B00C0837900752F038583307507
:1050A00031009000561203D51204E51203D5120503
:1050B0002F9000567A80E0A3F5F0E0A36C7005E530
:1050C000F06B6017DAF0D0830583740024C0E583A9
:1050D00034A550C1740512513AD322D083EA2AF57F
:1050E000F0E4C395F0F582124F9B78A0790A7A0616
:1050F00075F00FE3540FF652F00809DAF643F0F0BA
:10510000E5F004601D121BD7701BAB83AC821251FB
:1051100066EBB58306ECB58202C322740412513AE1
:10512000D322121BD7E5822582F582E5833583F5EC
:1051300083124FE0124FA90253DFF51A22C082C03A
:1051400083E583125850D083D082C082C083E58229
:10515000125850D083D08222C0E0782EE583F20826
:10516000E582F2D0E022C0E0782EE2F58308E2F595
:1051700082D0E02274001249E974001249E97400F7
:105180001249E974001249E974001249E922758351
:105190001B75821B75F040C0F0C082C083752F0163
:1051A0008583307531001203D51204E5D083D08297
:1051B000C082C083752F038582307531001203D5FC
:1051C000120583D083D08205830582D0F0D5F0C745
:1051D0007532FF7533FF227401F97418F8752F00CA
:1051E0007530007531001204767401F97419F87580
:1051F0002F017530D97531FF120476AC1812516643
:10520000E5822420F582E583347DF583C082C08366
:105210007401F9743BF8752F008583308582311253
:105220000476D083D0827401F97410F8752F00854C
:1052300083308582311203EF7810E2F5F0E518250E
:105240003BC395F0F518125166123C957853797C62
:10525000E2F72519F5190809E2F72519F519781665
:105260007953E2F3FA0809E2F32AFAC3E5199AF549
:1052700019125166123CBF125166E58275F008A4FE
:105280002420F582500205F0A8F0E58375F008A40B
:10529000282400F5837408F9747CF8752F00858341
:1052A00030858231120476787CE5187A082608DA8F
:1052B000FCF518789479007A0A75F00FE3540FF62C
:1052C00052F00809DAF643F0F0E5F0041257ED78F1
:1052D000A0790A7A0675F00FE3540FF652F0080928
:1052E000DAF643F0F0E5F0041257F57408F9747C2F
:1052F000F8752F00858330858231120420787CE593
:10530000187A08C39608DAFBF518125166C3E582CD
:1053100033F582E58333F583C3E58233F582E58394
:1053200033F583E5822400F582E583245BF583C0B1
:1053300082C0837404F9747CF8752F0185833085ED
:105340008231120476D083D0827404F97412F87515
:105350002F018583308582311203EF787C7912E545
:10536000197A0426F5F0E3C5F0C395F00809DAF3DD
:10537000F5197401F97418F8752F0075300075313E
:10538000001204207401F97419F8752F017530D9D1
:105390007531FF12042075831B75821B75F040C0A8
:1053A000F0C082C083752F038583307531001203EE
:1053B000D51204E5D083D082C082C083752F0185C9
:1053C00082307531001203D5120583D083D0820557
:1053D000830582D0F0D5F0C77532FF7533FF2212F6
:1053E0004FC5E5828583F0124FB7C39582C0E0E5D3
:1053F000F09583D0F045F07002C32250030254FAB6
:10540000124FC5C0E0C3E58224FEF582E58334FF78
:10541000F583D0E0124FA9E5828583F0124FB7B52E
:105420008207E5F0B58302C322124FB7AF83124F54
:10543000C5EFB58310AE8290002E787CE0F6A3080D
:10544000E0F602545D7EFE8F8305837402F9747C5E
:10545000F8752F0385833075310012047679007555
:105460002F038F307531009000561203D51204E5DA
:105470001203D512052F8F83758200124FB77D005E
:10548000E5836F7002AD82ED2456F582758300507E
:10549000020583C3EE9D20E05A03FCC082C083A3B3
:1054A000A3E0FAA3E0FBD083D082EAF0A3EBF0A361
:1054B000DCE9EE2456F58275830050020583787C82
:1054C000E6F0A308E6F07900752F038F3075310000
:1054D0009000561203D512056F1203D5120583856D
:1054E0002F32853033124FC5EFB583030255CE0FEF
:1054F00002542E740812513AD322124FB7AF8312BE
:105500004FC5EFB58310AE8290002E787CE0F6A3F5
:1055100008E0F602552E7E008F8315837402F9741D
:105520007CF8752F038583307531FE12047679007F
:10553000752F038F307531009000561203D5120479
:10554000E51203D512052F124FB77DFEE5836F706C
:1055500002AD82ED2456F58275830050020583C3A7
:10556000ED9E20E06B03FCC0E0C3E58224FEF582E3
:10557000E58334FFF583D0E0C082C083E0FAA3E086
:10558000FBA3EAF0A3EBF0D083D082DCDAEE245662
:10559000F58275830050020583787CE6F0A308E667
:1055A000F07900752F038F3075310090005612038B
:1055B000D512056F1203D5120583852F328530333E
:1055C000124FC5EFB583030255CE1F0254FFC3220D
:1055D000740912513AD3221249D0F5831249D0F5F9
:1055E000821249D070101249D0700BAF371249D0D7
:1055F0006F70030255F9024BF8C01EC01F85831E51
:1056000085821F1218A47401F9747CF8752F007537
:105610003000753100120476787CE6C3951EC39580
:105620001FD01FD01E251E251FF67401F9747CF8AB
:10563000752F00753000753100120420124A1102D6
:105640004AFB1249D0F583AF371249D06F70A712C9
:1056500086C61286C61286C61249F4E5361249E994
:1056600074001249E9E51A1249E974001249E97413
:10567000001249E974001249E974001249E9E5375A
:105680001249E93099FD024AFB905691C082C083CD
:10569000327581D375D000026466C082C083E58212
:1056A0002420F582E583347DF5837401F9743BF899
:1056B000752F00858330858231120420D083D082FB
:1056C000C082C083E58275F008A42420F5825002D0
:1056D00005F0A8F0E58375F008A4282400F583748C
:1056E00004F9747CF8752F008583308582311204AB
:1056F00020A3A3A3A37404F97480F8752F008583F5
:1057000030858231120420D083D082E582458360C7
:105710000EE5822418E58334FC74FFF5F0500BC0CD
:1057200082C083123CBFD083D08222120949C0E0DC
:105730007401F9747CF8752F007530007531001212
:105740000476787CE6D0F0C395F0F67401F9747CA9
:10575000F8752F0075300075310012042022753B5A
:10576000007854E4F2787C75F00876FF08D5F0FAFA
:1057700022751E30751F30C25AC25B75F005C0F02D
:10578000D2A3C251C2A2D254D2A1C253D2A4C252F5
:1057900012575E12216DD0F0204B09204C06D5F037
:1057A000DD0257E812580D403F1200D77881E6B469
:1057B000FF05C32275F005C0F012216DD0F0204C1A
:1057C00006D5F0F30257E8E53CB4021C78A0E624C5
:1057D000F6401508E624F6400F78A0E62430F51EC2
:1057E00008E62430F51FC3221200ABD32278947947
:1057F0007C7A05800678A079817A03E608540FC484
:10580000F5F0E608540F45F0F709DAEF22204B31A6
:10581000304C3AE53C600624FD24FC40301257F53C
:105820001200E475F005C0F0122169D0F0204B1190
:10583000203F06D5F0F002584D121262B40B0E80D4
:10584000031257ED753B007854E4F2C322D32222B1
:1058500022781FE254C07078E275F00A84C445F0E3
:10586000787EF6781EE254C07066E275F00A84C451
:1058700045F0787FF6781DE254E07054E275F00A46
:1058800084C445F07880F6781CE2604454E07040AF
:10589000E275F00A84C445F0C0E0781AE2030354CC
:1058A000C0D0F045F07881F6781BE2602354F070A8
:1058B0001FE275F00A84C445F0C0E07820E254F895
:1058C000700EE2C42354E0D0F045F07882F6C32293
:1058D000D32290000075F019C0F07402F9747CF8BE
:1058E000752F01858330858231120476787DB6FF6D
:1058F00002801318E551300C0AB4FF0788F0785580
:10590000E2A8F0666011E5822410F582500205835A
:10591000D0F0D5F0C3C322D0F0A3D322300C4DE594
:105920008224FFF582E58334FFF58375F019E58263
:105930002480E58334FE5005900000800AE582242F
:1059400010F58250020583C0F07402F9747CF8757A
:105950002F01858330858231120476787DB6FF026F
:10596000800518E6B55107D0F0D5F0C2C322D0F0BB
:10597000A3D322120114300C0C1258D2400390FF12
:10598000F112591C22C0511259A3D05122300C13CC
:105990001258D2400390FFF112591C5005F55112D4
:1059A00059D522E55170057551108023B410057545
:1059B0005111801BB411057551208013B420057559
:1059C00051FF800BB4FF0575510080037551FF1224
:1059D0005A86E551222230130CC213125851400549
:1059E00012679680031267E47881E6C45403E65494
:1059F0000F7882E6C45401E6540F7880E6C4540F51
:105A0000E6540F787FE6C4540FE6540F22300C0A98
:105A10001258D250051259D58003125A8622C2ACB0
:105A2000126296C2AC1286C61286C6D299C2B674EB
:105A3000FF1249E975370074421249E9746212494C
:105A4000E974151249E9742A1249E9741B1249E9EB
:105A500074001249E974001249E974001249E974AA
:105A6000001249E912030575F010C0F074001249E4
:105A7000E9D0F0D5F0F4E5371249E93099FDC24A92
:105A8000D2B61262962222201601227475787A12FA
:105A9000012F501C205F1BD25F125F50741A543FBD
:105AA0004400C2AF7518C075190BF51A120A3F22CF
:105AB000C25F1267E4203104203235227880E65438
:105AC0003FF5F07970E365F0702309E3787F667045
:105AD0001C203318D233125F50741A543F4400C252
:105AE000AF7518C075190BF51A120A3F2230323102
:105AF0007880E6543FF5F07972E365F0702309E3AE
:105B0000787F66701C203318D233125F50741A5499
:105B10003F4400C2AF7518C075190BF51A120A3F41
:105B200022C23322C2AC120A7D600CF51888191209
:105B30000DF1120A9580EFD2AC227E007F88900092
:105B40000075F000E49325F0F5F0A3C3E5829EE52F
:105B5000839F40F0E5F070022200E5F0C0E0E583AD
:105B6000125850E582125850D0E0125850C2ADC2BF
:105B7000ACD218D2A3C251D2A2C254C2A1C253D233
:105B8000A4C252C2A080EC300C417400788A120189
:105B90003E40387F087E007478787A12012FCE1349
:105BA000CE05E0DFF420190F7400789A12013E5000
:105BB00006EE78CD666014EE78CDF6F551C2AF757D
:105BC00018C075190485511A120A3F22C2AFF51A7E
:105BD00075190F751810020A3F22300CFC2057F976
:105BE0007401788A12013E40F07477787A12012F9E
:105BF000E492E0C0E07476787A12012FD0E033FEB0
:105C000020190F7401789A12013E500678D0E66E82
:105C100060C7EE78D0F620E10630E028025C57300D
:105C2000E014A259725850B1C259C258125EB074F1
:105C3000F8125BCC80A3D259C258125EB074F7122E
:105C40005BCC809520580ED258C259125EB0D25605
:105C500074F6125BCC8082A228825840F8D258C2D7
:105C600059125EC474F5125BCC025BD9C082C0834A
:105C7000D083D0822222303E09C2A3C251D2A4C214
:105C80005222D2A3C251C2A4C25222200C012274B9
:105C900074787A12012FE492E0C0E07473787A127B
:105CA000012FD0E092E1F5F0657A53F00385F07AA8
:105CB0006009E5F00303441A1286137472787A12AD
:105CC000012FE492E0C0E07471787A12012FD0E0E5
:105CD00092E1F5F0657B53F00385F07B6009E5F018
:105CE0000303441A12862922C2B6753700740312C0
:105CF00049E9E51E1249E9E51F1249E9744E1249C6
:105D0000E974081249E974011249E974061249E973
:105D10007848E2F5F0E5F01249E908E2F5F0E5F03F
:105D20001249E9784AE2F5F0E5F01249E908E2F5AE
:105D3000F0E5F01249E92442F8E2784CE2547FF5AC
:105D4000F07844E2C36001D3E5F092E7F5F0E5F0C6
:105D50001249E975F000E5F01249E9E5371249E921
:105D60003099FD22C2B6126CED126C7C753700744E
:105D7000031249E9E51E1249E9E51F1249E9744E8B
:105D80001249E9740C1249E974001249E9740A12C3
:105D900049E9C082C083A3A3A3E49375F064A4C0BF
:105DA000E0E5F01249E9D0E01249E9A3A3A3A3E496
:105DB0009375F064A4C0E0E5F01249E9D0E012491F
:105DC000E9D083D082E4931249E9A3E4931249E92C
:105DD000A3A3A3E4931249E9A3E4931249E9E58D4F
:105DE0001249E9E58B1249E9E5371249E93099FD95
:105DF00022C2B61212FCC0E075370074031249E9E2
:105E0000E51E1249E9E51F1249E9744E1249E97489
:105E1000041249E974021249E974021249E978ACA2
:105E2000E2F5F0E5F01249E9D0F0E5F01249E9E5D4
:105E3000371249E93099FD22C2B612127CC0E075D2
:105E4000370074031249E9E51E1249E9E51F1249BA
:105E5000E9744E1249E974041249E974021249E9DD
:105E600074021249E978ACE2F5F0E5F01249E9D0A4
:105E7000F0E5F01249E9E5371249E93099FD22C011
:105E8000F088F0C0F0C2AF7570007850E2F54BF5C5
:105E9000F008E2F54CD2AF45F0D0F0A8F0D0F070A9
:105EA00009B228202804125EBA22D2287570032273
:105EB000C2AF754BFF754CFFD2AF757000C20DC2FB
:105EC00028D2A722125E7FD256D25022C265027219
:105ED000B7D2650272B7305814202811543F4400DD
:105EE000C2AFF51A7519087518C0020A3F22D2B25E
:105EF000C2B4D293C322D2B2C2B4D2931286AE201D
:105F0000B2ECC2931286AE30B2E4D2931286AE12D5
:105F100086AE20B2D9C2931286AE1286AE30B2CE11
:105F2000D2B2C2B4D293D3221204C1C28474541226
:105F300004CCE412049B1204AEF5F06448255B33F4
:105F4000F55BE5F0255CB2E003F55CD9E9D284228B
:105F50007583DD75F010752F03858330753100C0B2
:105F600083C0F01203D51208DBD0F0D0830583D5AF
:105F7000F0E47532FF7533FF75710075720022E52C
:105F8000822400C0E0E58334DDF8D0E0C322C08283
:105F9000C0837401F9747CF8752F03858330858282
:105FA00031120476787CB6020CE57224FFF572E5B6
:105FB0007134FFF571D083D08222125F7FC082C01E
:105FC00083F5828883125F8E787C76007401F97481
:105FD0007CF8752F03858330858231120420D083AD
:105FE000D08222125F7FC082C083F5828883C08204
:105FF000C0837401F9747CF8752F03858330858222
:1060000031120476787CB60209D083D082D083D056
:106010008222E5722401F57250020571D083D0828C
:10602000787C76027401F9747CF8752F03858330CF
:10603000858231120420D083D08222125F7FC082F9
:10604000C083F5828883125F8E787C76017401F9B3
:10605000747CF8752F03858330858231120420D03B
:1060600083D08222125F7FC082C083F58288831230
:106070005F8E787C76037401F9747CF8752F038544
:106080008330858231120420D083D08222125F7F38
:10609000C082C083F58288837401F9747CF8752FFF
:1060A00003858330858231120476787CE6B4010260
:1060B000800CB402028007B4030280027400D08313
:1060C000D082221204C1C28474541204CCE412049B
:1060D0009B1204AEB40205755B018002D9F3D28431
:1060E00022755B007583DD75F00F752F0385833096
:1060F000753100C083C0F01203D51204E51203D538
:1061000079001260C3D0F0D0830583E55B7026D59B
:10611000F0D8752F038583307531001203D5120432
:10612000E51203D579A01260C37532FF7533FFE520
:106130005B7002D322C322E572457160167867E274
:10614000F5F008E245F0600BD37868E2957218E24A
:10615000957122C322C28C758A45758C5DD28CB232
:106160000020000132C000C001C0D0C0E0C0F07506
:10617000D008D24F121261126277051DE51D20E092
:106180000C20E10930181AE51D541F60592018042D
:10619000E54A6002B2B5D0F0D0E0D0D0D001D00056
:1061A00032205405A228B392A2E51D30E2031270FA
:1061B00013E51D541F7032D250C26978ABE2D5E0AE
:1061C00006D268D269743CF2C082C083126E94D049
:1061D00083D082E4B54648B5485AB56062B5696374
:1061E000B57867B57968B54969E4B54A43B547718B
:1061F000B54472B54D76B57077E54C454B601DE5FD
:106200004C2401F54C5002054B454B700FC20D203C
:10621000570A205807125EBAD256D25002618DD565
:1062200046B5C20D7548B4757700D242D24580A7F5
:10623000154A80B9D548A3C240C241C242809B15CD
:1062400060809AD5699AC26780961578809515798D
:106250008094D5499475450330180302568902612C
:10626000DA1547808BD5448BD2498087154D8086BF
:10627000D57086C2A78082E51DA2E330510292A3A9
:1062800030540292A230530292A122C2B6204A0296
:10629000D2B61262963275C800C2ADC2AC75CBFFE1
:1062A00075CA9875CDFF75CC98759853C298C299E8
:1062B000D2ACC2BC75C8347599062275C800C2AC90
:1062C000C2AD75980075CC2B75CDEBD2AD75C804F9
:1062D0002275C800C2ACC2AD759800E58A242BF5C2
:1062E000CC540F658C24EBF5CDD2AD75C80422C219
:1062F000A8C2AAC289C28BC2ACC2A9C2AB758F01A7
:106300001205C4D218125ED1125EB0E4F53B785487
:10631000F2787A75F010F2D5F0FCC257C258C25923
:10632000753DFF753FFF751D04C23FC240C241C2AB
:1063300042754801754900C245D24F756D00C233A0
:10634000C21AC21BD249C24A754410E4F540F54155
:10635000F542F534F536121EE0751E00751F80E417
:10636000F546F54FF54EF555F556F53EC225C226D4
:10637000C227C2037437785AF2785BF2785CF278FD
:106380005DF2D22175450375470178A87A0576FF3D
:1063900008DAFBC213781AE47A07F208DAFCC214AE
:1063A0007551FF78CDA651C215C20C757803756082
:1063B0001E756100C25EC211C212C20DC20EC20FB2
:1063C000C25AC25B755E00755D0075F0067842E4E6
:1063D000F208D5F0FB7948E4F309F3794AF309F3BD
:1063E000784CE4F212142A754AFAB2B57532FF7588
:1063F00033FFD25F7568007829740AF2126CCCC240
:1064000067756901756C1AC208C209C205C206C265
:1064100007D2A075700075710075720078AA74FAC1
:10642000F2E478B5F278B6F278B7F278AB743CF271
:10643000C26BC26AC266757700126E07C26CD26DFB
:10644000C26ED2701213EB758901758A3E758C5D30
:10645000C2B9D2A9D28CD2B6126296D2AFD293C2AE
:10646000B4D2B2B2B522C21875500375F0031286C9
:1064700096D5F0FAC25AC25B12245175500375F0DA
:1064800003128696D5F0FAC25AC25B1222ECC2AF52
:106490001213C102000020071320060820090D2056
:1064A0000802C32212143E1268D7D3221269E0D325
:1064B00022C27075F000C0F01274E4D0F0500343B3
:1064C000F008E5F022306A14203E2278B7E2306806
:1064D00006C268600214F224FA500922306B0E786A
:1064E000B7E27009E576540170031200E422C26B32
:1064F000C26AE478B7F222C2AF754AFAB2B5128620
:10650000AEB2B51286AEB2B5D2A07581D375D00049
:106510001262EF125C6C125B3A125F50121D04752E
:106520004AFA120CEF1264967550031225CF122509
:10653000E51200F1C2AF751880751904751A83123F
:106540000A3FD219300C0F120B0C125B87125BDA68
:10655000125A87125C8BC26FD2B7D2AFC218C2195F
:10656000000000D2B7D2AFC218C21900000020B795
:10657000091286AE20B703021D1E300C32120B0C1E
:106580001264C5E5745420601178AAE2D5E00A12BD
:1065900067E4125A1E78AA74FAF2E577600215775A
:1065A000300C0C125B87125BDA125A87125C8BE597
:1065B000616003D5610E126E001226CB1259D612FD
:1065C0005A0D800CD2A3C251C2A1D253D2A4C2523E
:1065D000E5607003125B24C254D2A1C253125C76F0
:1065E000C25AC25BD2567860E2600D24FD40097544
:1065F0006F021227C21264967861E2600D24FD409A
:1066000009756F031227C2126496E5735440600641
:1066100020A80312856D12216D204C08204B052007
:106620004D02801A302D09304106125C6C0266362C
:1066300012347F1264967829E215E0F27008782906
:106640007414F202656302659A0074A21266DEE8B1
:10665000126719E91267191267502274A21266DED6
:10666000E8126719E712671909D582F812675022F4
:1066700074A21266DEE812671974A31266DE12674E
:1066800039F709D5820412675022C296D2970000CA
:1066900000C29780E974A21266DEE81267191266DA
:1066A000A22274A31266DE126739F91267502274AF
:1066B000A27A08C296000000C297335005D2960213
:1066C00066C4C296D297000000C297DAEDD2960057
:1066D000D297000000309604C297C322D3227A08D2
:1066E000D296D297000000000000000000000000D9
:1066F00000000000C296000000C297335005D296F9
:10670000026705C296D297000000C297DAEDD296D2
:1067100000D297000000C297227A08335005D29623
:10672000026725C296D297000000C297DAEDD29692
:1067300000D297000000C297227A08D296C2970032
:10674000000000D297C3309601B333DAF0C297222B
:10675000C296000000D297000000D29622781079ED
:1067600084C082758205126670D0827884B6870EE6
:1067700008B6E00A08B6330608B6A902C322D32237
:1067800012675D400122787E760008760008760068
:10679000087601087601787C76000876007880E635
:1067A000543FF67800797CC08275820712665BD010
:1067B000821286967814797CC08275820712665B95
:1067C000D082128696788476870876E00876330839
:1067D00076A978107984C08275820412665BD082B3
:1067E000128696227802797EC082758205126670C2
:1067F000D082227882E603C4540775F018A4C0E062
:106800007880E6C4540375F00AA4F5F0E6540F2529
:10681000F0D0F025F075F03CA4C0F0C0E0787FE641
:10682000C4540775F00AA4F5F0E6540F25F0D0F033
:1068300025F0F5F0D0E03400C5F022206C56206041
:1068400021C0D0C0E0E8C0E0C0F0E54D7003856C29
:106850006A754D08D263126953D0F0D0E0F8D0E0E9
:10686000D0D0C28932206029C0D0C0E0E8C0E0C0EA
:10687000F0E54D7003756A00754D08A2B2B39263DE
:10688000126A38308502D205D0F0D0E0F8D0E0D0DE
:10689000D0C28B32C2A8C28932206CC9206026C007
:1068A000D0C0E0E8C0E0C0F0E54D7003856C6A75CB
:1068B0004D08C263126953308502D205D0F0D0E092
:1068C000F8D0E0D0D0C28B32C2A8C2AAC293C2B460
:1068D000C0E0128696D0E0C26CC293C2B4C289C234
:1068E0008BD2B2D2B3C260754D00856C6AC205C24C
:1068F000B8D288D2A8C2BAD28AD2AA22C26CC2A8FE
:10690000C2AAC289C28B22E56C141475F00884F502
:10691000F0C0F07830E230E002B26130E102B26102
:1069200030E202B26130E302B26108D5F0E7D0F0A4
:10693000E230E002B26230E102B26230E202B26200
:1069400030E302B26208D5F0E7206105306202C38D
:1069500022D322E56AB56C07A263926102699DB4F5
:106960000107A263926202699DC3E56C14956A40B7
:106970003275F004842430F8E205F0D5F006A26305
:1069800092E38016D5F006A26392E2800DD5F00660
:10699000A26392E18004A26392E0540FF2D56A02EE
:1069A000D26022856C6AD260227547321268C83084
:1069B0004F05C24F12027AE54760113060F1E56A77
:1069C000700A1268FC1269074002C3221268FCD3E5
:1069D00022C2A8C2AAC293C2B4C0E0128696D0E076
:1069E000D26CC293C2B4C289C28BD2B2D2B3C260DB
:1069F000754D00756A00C205C2BAD28AD2AA227544
:106A000047321269D1304F05C24F12027AE5476012
:106A10000C3060F1E56A70051268FCC3221268FC54
:106A2000D322C330E001B330E101B330E201B3302F
:106A3000E301B330E401B322E56A75F00584C0E0F8
:106A400024EED0E040552430F8E2A26392E503F250
:106A5000E56A700BE2541FB40B40756A05803B0574
:106A60006AE5F0B40434E2126A22502F540FF2188F
:106A7000E2540FB40F24D3E894307830F20404C009
:106A800082F58275F00B08E265F0F5F0D582F7D05B
:106A900082540F7006D260756A00221269E02201EA
:106AA0000000000000000000000A000000000000DC
:106AB00000000004060000000000000000080E03B3
:106AC00000000000000000000107020000000000BC
:106AD00000000A0608010000000000000402040F84
:106AE000000000000000080609080900000000007E
:106AF00000010E050F0500000000000A0C0A090B3A
:106B00000300000000040E0B000405020000000852
:106B10000E06070804070100000001050A040D081D
:106B20000E75F00A7994770009D5F0FA7830E2FA18
:106B300060400824F25007EA24F328F87A0DE25462
:106B40000FF26029EA1475F00AA4249FF5827400FC
:106B5000346AF583799D7E007B0AE493F5F0E2A424
:106B60002E2775F01084FEA7F0A319DBED08DACE0E
:106B7000C322D322094300A00954009F0966009E46
:106B80000977009D0989009C099B009B09AD009A2B
:106B900009BF009909D2009809E4009709F7009607
:106BA0000A0A00950A1D00940A3000930A430092D5
:106BB0000A5700910A6B00900A7F008F0A93008E9B
:106BC0000AA7008D0ABB008C0AD1008B0AE7008A55
:106BD0000AFE00890B1400880B2B00870B430086EC
:106BE0000B5C00850B7500840B8E00830BA7008265
:106BF0000BC100810BDB00800BF6007F0C10007EC8
:106C00000C2B007D0C47007C0C64007B0C81007A0F
:106C10000C9E00790CBB00780CDB00770CFB007637
:106C20000D1B00750D3B00740D5B00730D7D007234
:106C30000D9F00710DC200700DE4006F0E07006E15
:106C40000E2C006D0E51006C0E76006B0E9B006AD0
:106C50000EC100690EE900680F1100670F39006668
:106C60000F6100650F8900640FB300630FDE0062DF
:106C70001009006110340060105F005F7F42906B6C
:106C800074E493A3F5F0E493A3C3958BE5F0958D9D
:106C90005015A3A3DFEBE58224FFF582E58334FFE3
:106CA000F583E49314800BA3E493BF4205906B74C7
:106CB0008010C0E0E58224F9F582E58334FFF58396
:106CC000D0E02290006BE0A28733F02290006C7439
:106CD00000F090006B7455F090006D74FFF0900020
:106CE0006F7405F090006E7412F0D28122D286A2E9
:106CF000A4C0D0D2A475F000D5F0FDD5F0FDC28EB1
:106D000053890F438910758B00758D00C28FC2AFF8
:106D1000C2A4D28E208603308FFAC28E308F0675C1
:106D20008BFF758DFFD2AFD0D092A422F024FE400D
:106D300005308102C2812290006FE0D5E0EE7442FE
:106D4000F0126CEDD281E58B2499E58D34F240147C
:106D5000E58B24E1E58D34F3400EE58B24E0E58DF1
:106D600034FC400874158006741180027412FE9081
:106D7000006EE06E6015EEF0E5735404700DC2AF66
:106D80007518C07519008E1A120A3F22126CC36062
:106D90003B04603890006DE020E010D2E0F09000FD
:106DA0006CE070047405F022E4F02290006CE06066
:106DB0002E14F0702AE57354027024C2AF7518C007
:106DC000751900751A14120A3F026DDF90006DE00C
:106DD00030E00DC2E0F090006CE070CC743CF0222A
:106DE00090006CE060F914F070F5E573540270EFF8
:106DF000C2AF7518C0751900751A13120A3F80DFEB
:106E0000126D37126D8C229002EF75F008E4F0A33A
:106E1000D5F0FB9002F775F00874FFF0A3D5F0FBF6
:106E200022C0E0126E74D0E0B3502CC0E024F8D041
:106E3000E04022C082C083F5F024F7F582E43402FA
:106E4000F583E0C5F024EFF582E43402F583E5F044
:106E5000F0D083D082D322C0E024F8D0E04013C029
:106E600082C08324EFF582E43402F583E4F0D0831A
:106E7000D082C322C0E024F8D0E04016C082C08394
:106E800024EFF582E43402F583E0D083D0826002FF
:106E9000D322C3229002EF75F008E06003B4FF052F
:106EA000A3D5F0F62220E70414F080F43069F11441
:106EB000F0B480ECE4F080E8B440087400126E7422
:106EC000026F4AB441077401126E74807DB44207A8
:106ED0007402126E748073B443077403126E74806C
:106EE00069B444077404126E74805FB45407A274CA
:106EF0007275B38055B45506A274B075804CB45603
:106F000006A275B0748043B45706A2748275803AA5
:106F1000B45807A2727273B38030B45906A272B02B
:106F2000738027B45A06A273B072801EB45B06A2A7
:106F30007282738015C0E024E3D0E040132324B9AB
:106F4000C0E07400346FC0E022C3740122D380FA21
:106F5000E4C322A23EB380F2D250A26680EC80F05D
:106F6000A20D80E6A20F80E2A26E80DE80DF80E0CC
:106F7000A20E80D63067D280D4E571457260CA8097
:106F8000CC12613780C4A2597258B380BDA2588216
:106F90002880B7A258B02880B1A25980ADC3306A0A
:106FA00009203E0678B7E27001D3809EA265B380C7
:106FB00099C3E5786001D380918098809B80998007
:106FC00097809580938091808F8093809380958027
:106FD00097809980998099809B809E80A480A780CB
:106FE000AC80B080B480B680C380C680068010803C
:106FF0001D8018C3203E05E5796001D3026F4AC3A6
:10700000303E05E5796001D3026F4A026F50A270ED
:10701000026F4A12710D300C19C0E0C082C0837437
:1070200004120188D083D082D0E04003027048026D
:107030007032E538B40D0A302302802CD223D3807D
:1070400015126EB86022800EE538B40D06202303B9
:10705000027068C223C34009C229A229B392A58045
:1070600007D229A229B392A5300C19C0E0C082C072
:10707000837405120188D083D082D0E0400302706F
:107080009A027084E539B40D0A302402802CD2248F
:10709000D38015126EB86022800EE539B40D06203B
:1070A00024030270BAC224C34009C22AA22AB3929E
:1070B000A68007D22AA22AB392A6300C19C0E0C03B
:1070C00082C083740B120188D083D082D0E0400349
:1070D0000270EC0270D6E53AB40D0A300202802C40
:1070E000D202D38015126EB86022800EE53AB40D3C
:1070F0000620020302710CC202C34009C204A204AA
:10710000B392808007D204A204B3928022B21030DE
:107110001060E57454106003303E1BE57554047034
:1071200003204038E57554017003204111E5755482
:10713000027003204217C266754F00027172E54F5C
:10714000B401028024754F01754E40801CE54FB498
:1071500002028015754F02754EA0800DE54FB403F5
:10716000028006754F03754EF0E54E23F54EA2E002
:10717000926622C229A229B392A522D229A229B3BA
:1071800092A522B229A229B392A522F5F0030354B5
:107190003FB40258E53864086005E538B40D4AE5A7
:1071A000F089F0C0F0300C19C0E0C082C0837404D4
:1071B000120188D083D082D0E040030271D00271E6
:1071C000C1D0F0A9F05403B4020D1271730272B56C
:1071D000D0F0A9F00272B5B4010612717B0272B54B
:1071E000B403061271830272B50272B3B40362E58E
:1071F0003964086005E539B40DEFE5F089F0C0F0B9
:10720000300C19C0E0C082C0837405120188D0839D
:10721000D082D0E0400302722F02721CD0F0A9F09D
:107220005403B40211C22AA22AB392A60272B5D0A4
:10723000F0A9F00272B5B4010AD22AA22AB392A62A
:107240000272B5B40309B22AA22AB392A68066805C
:1072500062B4045FE53A64086005E53AB40D54E5AC
:10726000F089F0C0F0300C19C0E0C082C083740B0C
:10727000120188D083D082D0E04003027293027260
:1072800081D0F0A9F05403B4020FC204A204B39257
:10729000808022D0F0A9F0801CB40109D204A2049D
:1072A000B392808010B40309B204A204B392808028
:1072B000048000D322C322C0E07417306521B538A2
:1072C00007C229A229B392A5B53907C22AA22AB3B7
:1072D00092A6B53A07C204A204B39280D0E022B5C8
:1072E0003807D229A229B392A5B53907D22AA22AF2
:1072F000B392A6B53A07D204A204B39280D0E0229A
:10730000C0E01274D1D0E04023302C03203E1D2079
:10731000591AC0E0125ED6125EC4D0E020380BC20B
:10732000AF12863F751810120A3FD32220380BC2C5
:10733000AF12863F751820120A3FC322D20FC2AF88
:107340007518C0751900751A01120A3F30282620D9
:10735000582920360DC2AF754BFF754CF8D2AF12CD
:107360005EBA7852E2F546E576541060031242AAFE
:1073700078CE76FF2220340312744022C259C258BC
:10738000205709C0E0125EB0D0E0D256543F44C04E
:10739000C2AFF51A7519087518C0020A3FD259C252
:1073A00058205709C0E0125EB0D0E0D256543F4496
:1073B00080C2AFF51A7519087518C0020A3FD25875
:1073C000C259205709C0E0125EB0D0E0D256543FF7
:1073D0004440C2AFF51A7519087518C0020A3FD2A9
:1073E00058C259205709C0E0125EC4D0E0D25654AA
:1073F0003F4400C2AFF51A7519087518C0020A3F5C
:1074000030170122C0E074108004C0E0741178A02D
:10741000760A0875F00A84F608A6F0753C03D0E0F9
:1074200078B1F2087405F2D21722C20F754600C275
:1074300042C2AF7518C0751900751A02120A3F22B0
:10744000757700D2407548B4C2AF75185075190FE2
:10745000751AFF120A3F22C23ED270C2AF75186081
:1074600075190F751AFF120A3F757903C240C2439E
:1074700022D23EC270C2AF75187075190F751AFF0F
:10748000120A3F75790322C0E0125F50D0E0543FEA
:107490004400C2AFF51A75190B7518C0120A3F22C5
:1074A0007874F208F212269BC2AF7518C0751900E5
:1074B000751A50120A3F22400C305708C257205804
:1074C00003125EB0222057FC125ED6125EC4D25761
:1074D0002212784B400D127C49400812804740032D
:1074E00012844822127856400D127C5440081280B3
:1074F00052400312845322A290301E01B3785AE204
:1075000033F222106D030278F4301808C3785AE47D
:10751000F2027864E57554106003303EEF785AE269
:1075200060EF0460030278F220210320254FD2256A
:10753000300C19C0E0C082C0837400120188D0836F
:10754000D082D0E040030278F202754C7856E224F3
:10755000A4401CC082C083907793E225E00493F599
:10756000F0E225E093D083D082C0F0C0E0E222E2D6
:10757000C2AF751890751909F51A120A3F0278F210
:10758000125C761200D70278F2740112733C027812
:10759000F2740112730040E80278F2127457027814
:1075A000F2D267756905027570C0E07401126E2B26
:1075B000D0E0027570203E0320350CC0E074041248
:1075C0006E2BD0E00275700278F2743D027696025E
:1075D0007570C0E0E57654047005D0E0027570D097
:1075E000E00278F2C0E0D374011274B7D0E0027503
:1075F0007002757002757074001274000278F27473
:10760000101274000278F274111274000278F2748D
:10761000201274000278F27401F9747CF8752F005E
:1076200075308C7531F1120476787CE612740002A4
:1076300078F27401F9747CF8752F0075308C75310F
:10764000F1120476787CE612740A0278F2306B1E2E
:1076500078B6E2601978B7F27401543F4480C2AF43
:107660007518C0751909F51A120A3F02758002785B
:10767000F2306BFAE478B7F27401543F4440C2AF81
:107680007518C0751909F51A120A3F027580740140
:10769000127487027580203E061274710275801282
:1076A0007457027580E57354106007E41274A002E9
:1076B00075800278F2E5735410600874FF1274A0AC
:1076C0000275800278F2740112737C0278F2740100
:1076D0001273DF0278F274011273BE0278F2740141
:1076E00012739D0278F27400126E2B74011286E2FE
:1076F0000275807400126E5774011286F302758051
:107700007400126E7440EC0276E67402126E2B74F2
:10771000011287040275807402126E577401128779
:10772000150275807402126E7440EC02770A7403BD
:10773000126E2B74011287260275807403126E5725
:1077400074011287370275807403126E7440EC0264
:10775000772E303E0302769F0278F2203EFA0276C0
:10776000997400440112862902758074400277637F
:10777000748002776374C0027763740044011286D8
:1077800013027580744002777C748002777C74C029
:1077900002777C78F275897591759B757075707537
:1077A0007075A175A975B575CA757075CF75D275E7
:1077B000E47570757075707570757075707570752D
:1077C0007075707570757075707570757075707591
:1077D0007075707570757075707570757075707581
:1077E0007075707570757075707570757075707571
:1077F0007075707570757075F175F475F775FF7645
:1078000007760F76177632764D7671768E76967687
:10781000A576B576C676CE76D676DE76E676F3773C
:1078200000770A77177724772E773B77487570773C
:1078300052775B75707570757075707761776B775F
:10784000707775777A77847789778E7856E2B40B7C
:1078500003A22522C322203E097856E2B40D03A2DA
:107860002522C3222021062025030278F2C22530DA
:107870000C19C0E0C082C0837400120188D083D08C
:1078800082D0E040030278F202788B7856E260DA28
:10789000B4010612742A0278F2B402030278F2B438
:1078A0000305127471804BB40908203E363035331D
:1078B0008040B40A02743DB40D0BE5765404703276
:1078C000740D0278E3B40E0BC374011274B7740E16
:1078D0000278E3C0E024CED0E05008C0E024B0D06D
:1078E000E0500FC2AF7518A0751909F51A120A3FBA
:1078F0008000D26D22A291301F01B3785BE233F297
:1079000022106D03027CF2301808C3785BE4F202A7
:107910007C62E57554206003303EEF785BE260EFF7
:10792000046003027CF020210320264FD226300C75
:1079300019C0E0C082C0837401120188D083D08254
:10794000D0E04003027CF002794A7857E224A44058
:107950001CC082C083907B91E225E00493F5F0E2A5
:1079600025E093D083D082C0F0C0E0E222E2C2AF33
:1079700075189075190AF51A120A3F027CF0125C0C
:10798000761200D7027CF0740212733C027CF07411
:107990000212730040E8027CF0127457027CF0D2AD
:1079A0006775690502796EC0E07401126E2BD0E034
:1079B00002796E203E0320350CC0E07404126E2B59
:1079C000D0E002796E027CF0743D027A9402796E06
:1079D000C0E0E57654047005D0E002796ED0E00294
:1079E0007CF0C0E0D374021274B7D0E002796E026A
:1079F000796E02796E7400127400027CF0741012B9
:107A00007400027CF07411127400027CF074201275
:107A10007400027CF07401F9747CF8752F007530E5
:107A20008C7531F5120476787CE6127400027CF0D5
:107A30007401F9747CF8752F0075308C7531F5126E
:107A40000476787CE612740A027CF0306B1E78B6FD
:107A5000E2601978B7F27402543F4480C2AF7518DF
:107A6000C0751909F51A120A3F02797E027CF030BE
:107A70006BFAE478B7F27402543F4440C2AF751811
:107A8000C0751909F51A120A3F02797E7402127440
:107A90008702797E203E0612747102797E12745735
:107AA00002797EE57354106007E41274A002797EB7
:107AB000027CF0E5735410600874FF1274A0027920
:107AC0007E027CF0740212737C027CF074021273EA
:107AD000DF027CF074021273BE027CF07402127337
:107AE0009D027CF07400126E2B74021286E2027901
:107AF0007E7400126E5774021286F302797E74004F
:107B0000126E7440EC027AE47402126E2B7402124C
:107B1000870402797E7402126E577402128715026E
:107B2000797E7402126E7440EC027B087403126E4C
:107B30002B740212872602797E7403126E57740228
:107B400012873702797E7403126E7440EC027B2C2C
:107B5000303E03027A9D027CF0203EFA027A97744E
:107B600000440212862902797E7440027B6174808F
:107B7000027B6174C0027B617400440212861302AE
:107B8000797E7440027B7A7480027B7A74C0027BB7
:107B90007A7CF07987798F7999796E796E796E79B7
:107BA0009F79A779B379C8796E79CD79D079E2795F
:107BB0006E796E796E796E796E796E796E796E798D
:107BC0006E796E796E796E796E796E796E796E797D
:107BD0006E796E796E796E796E796E796E796E796D
:107BE0006E796E796E796E796E796E796E796E795D
:107BF0006E796E796E79EF79F279F579FD7A057A99
:107C00000D7A157A307A4B7A6F7A8C7A947AA37AD5
:107C1000B37AC47ACC7AD47ADC7AE47AF17AFE7BCD
:107C2000087B157B227B2C7B397B46796E7B507BD6
:107C300059796E796E796E796E7B5F7B697B6E7B2D
:107C4000737B787B827B877B8C7857E2B40B03A2B3
:107C50002622C322203E097857E2B40D03A2262231
:107C6000C322202106202603027CF0C226300C19F4
:107C7000C0E0C082C0837401120188D083D082D05A
:107C8000E04003027CF0027C897857E260DAB401BC
:107C90000612742A027CF0B40203027CF0B40305DD
:107CA000127471804BB40908203E36303533804061
:107CB000B40A02743DB40D0BE57654047032740DB1
:107CC000027CE1B40E0BC374021274B7740E027C12
:107CD000E1C0E024CED0E05008C0E024B0D0E050B5
:107CE0000FC2AF7518A075190AF51A120A3F800065
:107CF000D26D22A292302001B3785CE233F22210DE
:107D00006D030280F0301808C3785CE4F2028060F2
:107D1000E57554406003303EEF785CE260EF04604C
:107D2000030280EE20210320274FD227300C19C0F8
:107D3000E0C082C0837402120188D083D082D0E078
:107D400040030280EE027D487858E224A4401CC023
:107D500082C083907F8FE225E00493F5F0E225E076
:107D600093D083D082C0F0C0E0E222E2C2AF7518A7
:107D70009075190CF51A120A3F0280EE125C761209
:107D800000D70280EE740312733C0280EE7403127B
:107D9000730040E80280EE1274570280EED26775DD
:107DA0006905027D6CC0E07401126E2BD0E0027D8B
:107DB0006C203E0320350CC0E07404126E2BD0E022
:107DC000027D6C0280EE743D027E92027D6CC0E00A
:107DD000E57654047005D0E0027D6CD0E00280EEC0
:107DE000C0E0D374031274B7D0E0027D6C027D6CE6
:107DF000027D6C74001274000280EE741012740024
:107E00000280EE74111274000280EE74201274006D
:107E10000280EE7401F9747CF8752F0075308C7552
:107E200031F7120476787CE61274000280EE740159
:107E3000F9747CF8752F0075308C7531F712047663
:107E4000787CE612740A0280EE306B1E78B6E2602F
:107E50001978B7F27403543F4480C2AF7518C075E7
:107E60001909F51A120A3F027D7C0280EE306BFA86
:107E7000E478B7F27403543F4440C2AF7518C0753C
:107E80001909F51A120A3F027D7C740312748702E5
:107E90007D7C203E06127471027D7C127457027D37
:107EA0007CE57354106007E41274A0027D7C0280AC
:107EB000EEE5735410600874FF1274A0027D7C021A
:107EC00080EE740312737C0280EE74031273DF027F
:107ED00080EE74031273BE0280EE740312739D026F
:107EE00080EE7400126E2B74031286E2027D7C74A5
:107EF00000126E5774031286F3027D7C7400126EBA
:107F00007440EC027EE27402126E2B74031287043A
:107F1000027D7C7402126E577403128715027D7CF9
:107F20007402126E7440EC027F067403126E2B749E
:107F300003128726027D7C7403126E577403128726
:107F400037027D7C7403126E7440EC027F2A303E4F
:107F500003027E9B0280EE203EFA027E957400446E
:107F600003128629027D7C7440027F5F7480027F49
:107F70005F74C0027F5F74004403128613027D7C2D
:107F80007440027F787480027F7874C0027F7880AA
:107F9000EE7D857D8D7D977D6C7D6C7D6C7D9D7D81
:107FA000A57DB17DC67D6C7DCB7DCE7DE07D6C7D7C
:107FB0006C7D6C7D6C7D6C7D6C7D6C7D6C7D6C7D79
:107FC0006C7D6C7D6C7D6C7D6C7D6C7D6C7D6C7D69
:107FD0006C7D6C7D6C7D6C7D6C7D6C7D6C7D6C7D59
:107FE0006C7D6C7D6C7D6C7D6C7D6C7D6C7D6C7D49
:107FF0006C7D6C7DED7DF07DF37DFB7E037E0B7EE5
:10800000137E2E7E497E6D7E8A7E927EA17EB17E1B
:10801000C27ECA7ED27EDA7EE27EEF7EFC7F067F63
:10802000137F207F2A7F377F447D6C7F4E7F577D73
:108030006C7D6C7D6C7D6C7F5D7F677F6C7F717FFD
:10804000767F807F857F8A7858E2B40B03A227224F
:10805000C322203E097858E2B40D03A22722C3228E
:108060002021062027030280EEC227300C19C0E031
:10807000C082C0837402120188D083D082D0E040D5
:10808000030280EE0280877858E260DAB4010612BB
:10809000742A0280EEB402030280EEB40305127467
:1080A00071804BB40908203E363035338040B40A25
:1080B00002743DB40D0BE57654047032740D0280E9
:1080C000DFB40E0BC374031274B7740E0280DFC0EA
:1080D000E024CED0E05008C0E024B0D0E0500FC281
:1080E000AF7518A075190CF51A120A3F8000D26DF1
:1080F00022A285300101B3785DE233F222106D03D4
:108100000284F6301808C3785DE4F2028461E575F4
:1081100054806003303EEF785DE260EF046003025C
:1081200084F420210320034FD203300C19C0E0C097
:1081300082C083740A120188D083D082D0E04003C9
:108140000284F40281467859E224A4401CC082C013
:1081500083908390E225E00493F5F0E225E093D04C
:1081600083D082C0F0C0E0E222E2C2AF7518907501
:10817000190DF51A120A3F0284F4125C761200D728
:108180000284F4740412733C0284F47404127300C5
:1081900040E80284F41274570284F4D267756905CA
:1081A00002816AC0E07401126E2BD0E002816A2065
:1081B0003E0320350CC0E07404126E2BD0E0028127
:1081C0006A0284F4743D0282930284F402816AC0DC
:1081D000E0E57654047005D0E002816AD0E00284C4
:1081E000F4C0E0D374041274B7D0E002816A028153
:1081F0006A02816A74001274000284F474101274AA
:10820000000284F474111274000284F47420127455
:10821000000284F47401F9747CF8752F0075308CB9
:108220007531F3120476787CE61274000284F474DB
:1082300001F9747CF8752F0075308C7531F31204D8
:1082400076787CE612740A0284F4306B1E78B6E20B
:10825000601978B7F27404543F4480C2AF7518C0F7
:10826000751909F51A120A3F02817A0284F4306BFB
:10827000FAE478B7F27404543F4440C2AF7518C0B2
:10828000751909F51A120A3F02817A74041274876B
:1082900002817A203E0612747102817A12745702AA
:1082A000817AE57354106007E41274A002817A02A7
:1082B00084F4E5735410600874FF1274A002817A8C
:1082C0000284F4740412737C0284F474041273DF65
:1082D0000284F474041273BE0284F4740412739D55
:1082E0000284F47400126E2B74041286E202817A06
:1082F0007400126E5774041286F302817A740012AD
:108300006E7440EC0282E37402126E2B74041287C6
:108310000402817A7402126E577404128715028166
:108320007A7402126E7440EC0283077403126E2B8F
:10833000740412872602817A7403126E5774041231
:10834000873702817A7403126E7440EC02832B30FB
:108350003E0302829C0284F4203EFA02829674005C
:10836000440412862902817A744002836074800278
:10837000836074C002836074004404128613028117
:108380007A7440028379748002837974C00283799D
:1083900084F48183818B8195816A816A816A819B62
:1083A00081A381AF81C4816A81C981CF81E1816A62
:1083B000816A816A816A816A816A816A816A816A65
:1083C000816A816A816A816A816A816A816A816A55
:1083D000816A816A816A816A816A816A816A816A45
:1083E000816A816A816A816A816A816A816A816A35
:1083F000816A816A81EE81F181F481FC8204820CC0
:108400008214822F824A826E828B829382A282B2EF
:1084100082C382CB82D382DB82E382F082FD830738
:1084200083148321832B83388345816A834F835848
:10843000816A816A816A816A835E8368836D8372DF
:10844000837783818386838B7859E2B40B03A203FD
:1084500022C322203E097859E2B40D03A20322C3AD
:10846000222021062003030284F4C203300C19C029
:10847000E0C082C083740A120188D083D082D0E029
:1084800040030284F40284887859E260DAB4010679
:1084900012742A0284F4B402030284F4B4030512B1
:1084A00074718050B40908203E3B3035388045B4A3
:1084B0000A02743DB40C02803BB40D0BE576540403
:1084C0007032740D0284E5B40E0BC374041274B7D9
:1084D000740E0284E5C0E024CED0E05008C0E02451
:1084E000B0D0E0500FC2AF7518A075190DF51A1273
:1084F0000A3F8000D26D22E5735440601AE574543F
:108500000270061274F7127503E5745404700612B3
:1085100078F5127901800C1274F71275031278F550
:10852000127901127CF3127CFF1280F11280FDC2DD
:108530002120450122C245C2AF7518C075190075CA
:108540001A54120A3F22E8C0E07856E26403601829
:108550007857E2640360117858E26403600A78593E
:10856000E264036003C38001D3D0E0F822E4A228D0
:1085700092E0A22992E1A22A92E2A20492E3F56E8D
:10858000756F051226117403500412279D221227BD
:1085900075788DE6C0E0E57454026012D0E0C0E06A
:1085A00054071285CBD0E0C0E054071285CBE574A8
:1085B00054046014D0E0C0E0C454071285EFD0E04A
:1085C000C0E0C454071285EFD0E022A225301E017E
:1085D000B34007D320E10A0285EEC320E2030285FF
:1085E000EE301E01B3E49400785AF212750322A211
:1085F00026301F01B34007D320E10A028612C320B0
:10860000E203028612301F01B3E49400785BF21299
:10861000790122A2E69272A2E79273C2AFF51A75AF
:10862000190D7518C0120A3F22A2E69274A2E792B1
:1086300075C2AFF51A75190F7518C0120A3F22B42A
:10864000010775190F751AE122B4020775190F7524
:108650001AE222B4030775190F751AE322B404074E
:1086600075190F751AE422B4110775190F751AD10F
:1086700022B4120775190F751AD222B4130775198F
:108680000F751AD322B4140775190F751AD42275F1
:10869000190F751AD422C28E53890F438910758B16
:1086A000D6758D97C28FD28E308FFDC28E22C28E2C
:1086B00053890F438910758BEB758DCBC28FD28E8A
:1086C000308FFDC28E22C28E53890F438910E58AF6
:1086D000C4242BF58B758DEBC28FD28E308FFDC2EB
:1086E0008E22543F4400C2AFF51A75190A7518C09E
:1086F000020A3F543F4480C2AFF51A75190A751833
:10870000C0020A3F543F4400C2AFF51A75190C75F8
:1087100018C0020A3F543F4440C2AFF51A75190C05
:108720007518C0020A3F543F4480C2AFF51A75194C
:108730000C7518C0020A3F543F44C0C2AFF51A7509
:10874000190C7518C0020A3F7401126E5774041296
:108750006E57220000000000000000000000000032
:108760000000000000000000000000000000000009
:1087700000000000000000000000000000000000F9
:1087800000000000000000000000000000000000E9
:1087900000000000000000000000000000000000D9
:1087A00000000000000000000000000000000000C9
:1087B00000000000000000000000000000000000B9
:1087C0000000000000000000000000000000505207
:1087D000343032207665722E3133312E312E3120F5
:1087E0004864773A482032342D31302D30352032EC
:1087F000333A31342020004352430000000000D5BA
:00000001FF
:0300000306028072
